:100200004F726967696E616C2046696C653A20704F
:10021000726F6A6563742E6865780D0A4F75747025
:10022000757420446174653A20323030392F30358E
:100230002F32330D0A4F75747075742046696C65E2
:100240003A206B6C3537632E68657800000000003B
:10025000000000000000000000000000000000009E
:10026000000000000000000000000000000000008E
:100270000000000000000000000000000000002658
:109769000D0A0D0A205B4B4C3537435D0D0A0D0A76
:10977900000D0A0D0A00557365204B4C35784220BF
:10978900494F20446566696E650D0A005573652069
:109799004B4C35784320494F20446566696E650D09
:1097A9000A00416C6C204F757470757420456E61A8
:1097B900626C650D0A00416C6C204F75747075748C
:1097C90020446973616C650D0A00028001010B0474
:1097D9000B0801020801070107020280004000107E
:0A97E9000020000100020004000847
:0C8C680041F9EF0041F907FF41F9FA0063
:10A5A70090FDD7E0FF7408A807082235F0FAEBF012
:10A5B700A3EAF0A3E9F02290FDD6E075F021A424E8
:10A5C7000DF582E434F9F583E022EF75F021A42438
:10A5D700082290FDD6E0FFC32290FDD6E004F022CA
:1051AA00E490FDD6F0A3F0A374FFF07F0512B13CA2
:1051BA00E4F520FB7D027F041267D27DFF7F051292
:1051CA0078E37B027DFF7F051267D27D027F04129E
:1051DA00936BEF600C0D7F0612777C7B027D038058
:1051EA000B7D0F7F0612777C7B027D0F7F0612678D
:1051FA00D2E4FB7D017F0A1267D2E4FB7D037F0CB8
:10520A001267D2E4FB7D047F061267D2D2AF75FF24
:10521A00387BFF7AB0790B12B148E4FF12A7917D6F
:10522A00017F407E02128FB87BFF7A97796912A3B9
:10523A00B17BFF7A02790012A3B17BFF7A97797A60
:10524A0012A3B17BFF7AB179B77F0312B16A7B00EF
:10525A007C077DD012006E7D027F0412936BEF7B78
:10526A00FF60117A97797F1255FB7497F074D31205
:10527A0055E780397A9779951255FB7497F074E35C
:10528A001255E77D0C7F0B1278E37B017D0C7F0BB7
:10529A001267D27D017F081278E37B027D017F08C5
:1052AA001267D21294047D017F0812777C7F011263
:1052BA00B13C7B017AF97908E4FD127F5D7AF979CC
:1052CA00297DB41255DF7AF9794A7DB9127F5D7A60
:1052DA00F9796B7DE01255DF7AF9798C7DE5127FD9
:1052EA005D7B017AF979AD7DE8127F5D7B017AF900
:1052FA0079CE7DED127F5D7B017AF979017D70129D
:10530A0090F97B017AF979037D7E1290F97B017A13
:10531A00F979057D7C1290F97AF979F07D60125558
:10532A00F37AF979F27DE0129C037AF979F47DE255
:10533A001255F37AF979F67DE4129C037B017AF926
:10534A0079F87DE6129C03E490FDD6F012A5D99473
:10535A00035054EF75F002A42401F974F935F0FAF8
:10536A007B01C003C002C001E012A5D2F974F99012
:10537A00FC6512A5B290FDD6E075F042A4FFAEF02E
:10538A002429F974F93EFA90FC6812A5B5744A2FDB
:10539A00F974F93EFAA312A5B5D001D002D00312CE
:1053AA0082F312A5E080A590FD6A7401F0A374F956
:1053BA00F0A37408F07B017AF979F012B05AE490FC
:1053CA00FDD6F012A5D994045033EF75F002A42447
:1053DA00F2F974F935F0FA7B01C003C002C001E0AA
:1053EA0075F021A4246BF974F990FD6A12A5B2D064
:1053FA0001D002D00312B05A12A5E080C6E4FFFE23
:10540A0012AFB4EFD39403E4400690FD9FF0800AF4
:10541A00FFFE12AFB490FD9FEFF090FD9F7401F074
:10542A002008030255D9C20890FDD67403F0E4A3FC
:10543A00F012A5D9940740030254F112A5D1F582BE
:10544A00E434F9F583E0FB703912A5BEFC30E40CB4
:10545A0012A5A78002C313D8FC0254D0EC30E5177A
:10546A0090F9EFE075F01484E5F0707112A5A78049
:10547A0002C313D8FC803E12A5A78002C313D8FC2E
:10548A008055EB6405601390FDD6E012A5D2F58233
:10549A00E434F9F583E0640C703412A5BE30E61DDD
:1054AA0090F9EFE075F02884E5F0703112A5A78035
:1054BA0002C313D8FCFD7F05126AAE802012A5A78D
:1054CA008002C313D8FCFD7F051278E3800F12A572
:1054DA00A78002C313D8FCFD7F0512777C12A5E0D2
:1054EA00A3E004F002543B90F9EFE004F0C394C83F
:1054FA004002E4F07B017AF9790812373190FDD63F
:10550A007401F012A5D99403501312A5D1F974F9B4
:10551A0035F0FA7B0112560612A5E080E690FDD618
:10552A007403F012A5D99407501312A5D1F974F98E
:10553A0035F0FA7B0112237412A5E080E6E520B467
:10554A000F0D7D027F0612777C7D017F06801C7D10
:10555A00027F061278E37B017AF9790112A97AEFC0
:10556A007D017F0660051278E3800312777C90F94B
:10557A0007E025E0F0E0FE7D047F0612936BEF6002
:10558A00047F0180027F00EE4FFF90F907F0BF7F92
:10559A000EE520B40F047F0980027F1212A0213089
:1055AA00090AC2097F0112AC8612A021123CE52029
:1055BA000D0302542A90F9FAE0FF04F0EFD3946441
:1055CA00500302542AC20D7F0912A02102542A4311
:1055DA00870102542A7B01127F5D7B0122A3F07BA3
:1055EA00017AF8790012A9AC227B01129C037B0193
:0C55FA002212A3B190FD6474FFF0A32204
:10A02100EF24EE602E240970547BFF7A9779AB12EE
:10A03100A3B1E4F5207B017AF9796B12B15F7AF96A
:10A04100798C12B15F7AF979AD12B15F7AF979CE73
:10A0510002B15F7BFF7A9779BF12A3B175200F7BA5
:10A06100017AF9796B12B1547AF9798C12B1547A77
:0EA07100F979AD12B1547AF979CE12B15422B8
:10B00B00AE07E4FF12AC86BF8609EE7006EDB410F6
:04B01B0002D2092232
:03B1B700D2082299
:104238000000000000000000000000000000000076
:104248000000D60980A020E02D101060A200040311
:10425800000000188C0AD08A20E02D10103E96002D
:104268000403000000188C0AD08A20E02D10103EAC
:104278009600100900000018011D007251D01E2080
:104288006E28550010090000001E011D8018711CC1
:104298001620582C250010090000009E8C0AA01436
:1042A80051F01600267C43000403000000988C0A95
:1042B800A01451F01600267C430010090000009855
:1042C8008C0AA01451F01600267C43000403000059
:1042D80000188C0AA01451F01600267C430010091F
:1042E8000000001818154028B2F016004CF84300DA
:1042F80004030000009818154028B2F016004CF886
:10430800430010090000009818154028B2F0160064
:104318004CF8430004030000001818154028B2F0B8
:1043280016004CF843001009000000181815A014D6
:1043380051E02D10207C9600040300000018181589
:10434800A01451E02D10207C9600100900000018E0
:10435800023A801871382D40582C45001009000089
:10436800001E8C0AD090204031200C4055000403D8
:10437800000000188C0AD090204031200C405500D5
:10438800100900000018011D00BC52D01E20B828DA
:10439800554010090000001E011D80D0721C162017
:1043A800102C258010090000009E8C0AA0205120A6
:1043B8001810187E23000403000000988C0AA0201F
:1043C80051201810187E23001009000000988C0A4C
:1043D800A02051201810187E2300040300000018A4
:1043E8008C0AA02051201810187E23001009000004
:1043F800001818154040B220181030FC23000403A0
:104408000000009818154040B220181030FC230016
:1044180010090000009818154040B220181030FC10
:10442800230004030000001818154040B22018109B
:1044380030FC23001009000000181815A020514076
:1044480031201880550004030000001E1815A02014
:10445800514031201880550010090000001E023A12
:1044680080D072382D40102C458010090000001EA5
:10447800011D803E73382D407E2C458010090000B8
:10448800001E011D80D072382D40102C4580100967
:104498000000001E011D80D072382D40102C458070
:1044A80010090000001E3B2A4028B2E02D1060F8D9
:1044B80096000403000000183B2A4028B2E02D10A3
:1044C80060F89600100900000018302A4040B240F9
:1044D800312030005510040300000018302A4040F5
:1044E800B240312030005510100900000018201C7F
:1044F8008080711C552020A8750410090000009ABE
:10450800023A80D0721C1620102C25801009000059
:10451800009E023A00BC52D01E20B828554010090F
:104528000000001E1815D090204031200C40550086
:104538000403000000181815D090204031200C40CA
:1045480055001009000000181815D09020201810E8
:10455800187E23000403000000981815D09020202E
:104568001810187E2300100900000098023A8018DD
:10457800711C1620582C250010090000009E023AD4
:10458800007251D01E206E28550010090000001E30
:104598001D15D08A20E02D10103E9600040300005F
:1045A80000181D15D08A20E02D10103E9600100925
:1045B800000000181D15A01451F01600267C4300B9
:1045C8000403000000981D15A01451F01600267C65
:1045D8004300100900000098302AD0902040312074
:1045E8000C405500040300000018302AD0902040E9
:1045F80031200C405500100900000018302AA02076
:1046080051201810187E2300040300000098302A57
:10461800A02051201810187E2300100900000098CF
:104628003B2AD08A20E02D10103E9600040300009B
:1046380000183B2AD08A20E02D10103E9600100961
:10464800000000183B2AA01451F01600267C4300F5
:104658000403000000983B2AA01451F01600267CA1
:10466800430010090000009800FFFFFFFFFFFF0054
:104678001710010901000000000E01038073417842
:104688002A7C119E59479B271050540000000101B5
:104698000101010101010101010101010101011DE6
:1046A800007251D01E206E28550010090000001E0F
:1046B8008C0AD08A20E02D10103E960004030000DA
:1046C8000018000000FC0045502D48444D492D526B
:1046D800580A2020000000FD003B3D0F2E08000A6C
:1046E80020202020202001D402031D714A840513B4
:1046F8001401020311121023090707830100006542
:10470800030C001000023A801871382D40582C45CF
:104718000010090000001E011D8018711C16205889
:104728002C250010090000009E011D00BC52D01E5F
:1047380020B828554010090000001E011D80D072C5
:104748001C1620102C258010090000009E8C0AD011
:1047580090204031200C4055000403000000180050
:10476800000000000000001E097F070F7F071707E1
:10477800503F06C04D02005706005F7E01677E006D
:068C740041FD9F00C12F2D
:104CC30090FC06E0FBA3E0FAA3E02480F9E43AFABF
:104CD300EEFF7E0029F9EE3AFA121932FD90FC1923
:104CE300E0FBA3E0FAA3E0F990FC14E0F5827583FE
:104CF30000ED1219ACEF2481FFEE33FE90FC06E0C9
:104D0300FBA3E0FAA3E0F98F828E8312194BFF9085
:104D1300FC14E02401FDE433FC90FC19E0FBA3E068
:104D2300FAA3E0F98D828C83EF1219AC90FC0FE0AB
:104D330090FC062482FFE433FEE0FBA3E0FAA3E049
:104D4300222480F9E43AFA90FC0FE0FF7C0029F971
:104D5300EC3AFA121932541FFEEF2E90FC11F09028
:104D6300FC0EE004F0A3E004F090FC06A3E0FAA339
:104D7300E02480F9E43AFA90FC0FE022E92480F978
:104D8300E43AFAEE7E0029F9EE3AFA021932FF907C
:104D9300FDA1E02FFF90FDA0E03400FEE92FF9EA2A
:104DA3003EFA121932FF22F990008212194BC3FF07
:104DB30090FC0FE0FE9F22F98F828E8302194BF93C
:104DC3008D828C8302194B90FC13E0FF90FDA0E0D1
:104DD300FCA3E0FDC39F7480F8EC6480982290FCF0
:104DE3000F541F04FFE02FF02290FC0EE02480FFFD
:104DF300E433FE90FC092290FC0FE0FE90FC11EFDF
:104E0300541FFFEE2FF022FE04F0EE7C0029F9EC94
:104E13003AFAEF02199A90FC887401F0A374FCF03B
:104E2300A37414F090FC1CE0F9A3E0FAA3E090FC57
:104E33008BC9F0A3EAF0A3E9F022F97F807E001288
:104E4300190C90FC0D7401F022F990008212194B99
:104E5300FF90FC0EE0FE2290FC13F9E0FE04F08EBE
:104E630082758300EF0219ACFF90FD9EE02FF09056
:104E7300FDA1E004F022EE2480F582E433F58312F1
:104E8300194BFF54E02290FDA0E0FEA3E0FF229027
:104E9300FC0EE02480FDE433FC90FDA1E02DFD90A9
:104EA300FDA0E03CFC90FC09221219ACE490FD9EAD
:104EB300F090FDA0F0A3F022F990008312194B5457
:104EC300C0440190FC12F090FD1C7401F0A374FC2B
:104ED300F0A37413F090FC162204F0EE2480FDE49A
:104EE30033FC90FC092290FDA0E004F02290FC1317
:104EF300E0FFC390FDA1E09F7480F890FDA0E06403
:104F0300809822FF7C0029F9EC3AFA021932FF90CB
:104F1300FC14E02402FDE433FC90FC1922E429F99B
:104F2300EA3401FA12193254FE12199A90FC06223D
:104F3300F9EF9000010219AC90FC0FE004F0E0FFE0
:104F43007E0090FDA0EEF0A3EFF090FC0FF0229016
:104F53000023F912194BFF90FC0922F98D828C83EF
:104F6300EF0219ACFF04F07E00E92F22900002F952
:104F730012194BFF90FC0622EF541FFFEE2F90FCFB
:104F830010F022541F04FF90FC0EE02FF02290FC3F
:104F93000F7404F022F990007E02194B9000017403
:104FA3000C1219ACE49000020219AC90FC11E0FF62
:104FB30090FC0FE02290FC0FE0FF7E0090FDA0E04C
:104FC300FCA3E0FD2FFFEE3CFE90FC11E0FBD3EFD2
:104FD3009B7480F86E9822541FFF90FDA1E02FF080
:104FE30090FDA0E0340022E429F9EA3401FA021921
:104FF30032541FFEEF2E90FC11F090FC0EE004F0F3
:1050030022547FFFEE2480FDEC33FC90FC092290B8
:10501300FC0EE0FF7E00ED2FFFEE3CFE90FC10E067
:10502300FDD3EF9D74806E982290FC0EE02480FFE8
:10503300E433FE90FDA1E02FFF90FDA0E03EFE9043
:10504300FC092290FC0FE004F022FD7C00EF2DFD13
:10505300EC3EFCE92DF9EA3CFA021932F9EF900033
:10506300020219AC90FC0E7404F02274802DF582B8
:10507300E43CF58302194BC3947FEE648094802251
:1050830090000374101219ACE49000040219AC24CC
:1050930080F9E43AA801FCAD032290006F12194B8A
:1050A30064FD2290FC14F9E0F58275830022C39419
:1050B30005EE648094802290FC0EE02480FDE433AE
:1050C300CD2FFFED3EFE90FC0922FF90FC0EE02465
:1050D30082222FF582E43EF58302194B90FD9EE078
:1050E30014F4FF222480F9E43AFA22F990008202B0
:1050F300194BF990010002194BF990006C02194BFE
:1051030090FC14E02403F022F990007E740102194C
:10511300ACC390FC15E094052290FC0EE0FF7E00EA
:105123002480FDEE33FC22F9900001E41219AC90C7
:105133000002E42290FD9FE064032290006D0219B7
:105143004B90006E02194BFC8D82F58302194BF9CB
:1051530090002302194BF990002402194BF9900097
:105163002502194B90FC0FE02403F02290FC10E081
:10517300FF90FC0EE0D39F2290FC0EE02403F0226C
:10518300EF2481FFEE33FE90FC0922A3F0A3EBF0A2
:10519300A322F8AC02AD03A32212199A90FC1F229A
:0751A300F912224E7E0022EA
:1092350090FDD9EB124E3590FDD9124D3CF9EA4916
:109245004B70030292D090FDD9124D3CF8AC02ADA3
:10925500037BFF7A4679707E017F0012190C124E4E
:10926500AF124E8912507A501390FDD9124D3C120F
:109275004DBA124E6B70EA124EE980E51250DF903E
:10928500FDD9124D3CF990007FEF124EAC124E897C
:1092950012507A501690FDD9124D3C1250E7124DDE
:1092A5009F124E6C70E7124EE980E21250DF90FD7E
:1092B500D9124D3CF99000FFEF1219AC124FEA4458
:0C92C5000112199A440212199AC22F22B9
:1095C30090FDDCEB124E3590FDDC124D3C124F98B2
:1095D3006401707690FDA0F0A37404F090FDDC129A
:1095E3004D3C1250EE124DCE504F12506E54E0646B
:1095F30060701F748112507064037032124E89249C
:10960300821250D6640C702674831250D5701F7F5B
:10961300012290FDDC124D3CF990FDA1E02480FF76
:10962300124FE38F82F58312194B124FDAF0124E69
:109633007270A9124EE90295DF90FDDC124D3C12C7
:0D96430050EE124EF440037F00227F002203
:109DC60090FDDFEB124E3590FDDF124D3C124F98A1
:109DD600C39401404E90FDA0E4F0A37404F090FDFE
:109DE600DF124D3C1250EE124DCE502112506EFB3A
:109DF60054E0FFBF6008ED2480FFE43CFE22EB1236
:109E06004FDAF0124E7270D6124EE980D190FDDF15
:109E1600124D3C1250EEFFC3ED9F7480F86C9840D3
:079E2600028000E4FEFF22B0
:10A9DD00748112199A7402124F357403124FA89094
:10A9ED00000374111219AC741212508C900005747E
:10A9FD00041219AC90FD1C124D3CF9740602199A03
:10A83900740912199A90000174071219AC7407125D
:10A84900506190FC88124D3CF9740312199A90FCDE
:10A859008B124D3CF9740112199A90FC8B124D3CE4
:06A8690012512A0219AC95
:10AF9D00740312199A124F9F12508390FD22124D75
:07AFAD003CF9740502199A3A
:10A5640090FC8EEB124E3590FC8E124D3CF8AC02F2
:10A57400AD037BFF7A4779707E007F1812190C9027
:10A58400FC91124D3CF9741812199A90FC94124DD6
:10A594003CF9744F12199A90FC94124D3C12512AB2
:03A5A4000219ACED
:1002800090FC06EB124E35E490FC0DF07B0190FCE7
:100290001604F0A374FFF0748012518E74FFF07492
:1002A0009E12518E74FFF0A374CBF0A3EBF0A374F5
:1002B000FFF0A374CEF090FC06124D3CF9EA494BD6
:1002C0007002FF2290FD9FE0640260030203BF9072
:1002D000FC06124D3C1250F520E0030217AD124F00
:1002E00020124D3C125195124D3C124E3D90FC098E
:1002F000124D3C124F98640160030217AD90FC064A
:10030000124D3C1250F520E1030217AD124FEA5492
:10031000FD12199A90FC09124D3C1250E7C003C01F
:1003200002C00190FC06124D3C125092D001D00246
:10033000D003124E3E90FC0CE030E0030217AD12E9
:100340004F9190FC06124D3C124DAA40030217AD8E
:10035000124D7FFF54E064607053EF541FC3940745
:1003600050030217AD125046E0FF2485FDEE33FC2A
:1003700090FC06A3E0FAA3E0125057548F12519C50
:10038000124D3CF990000612194BFDC3941E500209
:1003900080027D1EEF2486FFE43EFE90FC06124D97
:1003A0003CF98F828E83ED1219AC0217AD90FC06DA
:1003B000124D3C124D74124D87124DE102034290D2
:1003C000FC09124D3C124F98D3940140037F002248
:1003D00090005A12194B707890005B12194B707094
:1003E00090005C12194B706890005D12194B64FD0F
:1003F000705E124EB4124E89C39412EE64809480E3
:10040000504E90FC09124D3CF9EF245AFFE43EFE99
:100410008F82F58312194B90FC12F090FDA1E0241D
:100420006CFD124FE312514B8F828E831219AC90E8
:10043000FC12E0FF90FDA1E0246CFD124FE38D82E1
:10044000F583EF1219AC124E7270AA124EE980A514
:1004500090FC06124D3C1250F530E00F124F201266
:100460004D3C125195124D3C124E3D1251376003D6
:1004700002052E90FC06124D3C124F52124D3C12BA
:1004800051524F4421FF90FC16124D3CF9EF124F90
:100490002C124D3C900024124F55124D3C125159D4
:1004A0004F4408FF90FC16124D3C124F3390FC064F
:1004B000124D3CF9900025124F56124D3C125160DE
:1004C0004FFF90FC16124D3C12505F90FC09124DEC
:1004D0003C1250FC60030205FA12513E6003020513
:1004E000FA12514460030205FA12509D600302059E
:1004F000FA90FC06124D3C1250FC60030205D21229
:10050000513E60030205D2125144701F12509D707B
:100510001A900075124F56124D3CF9900075121941
:100520004BD39F50030205FA0205CF0205D290FC7F
:1005300006124D3C124F52124D3C1251525F442153
:10054000FF90FC16124D3CF9EF124F2C124D3CF966
:10055000900024124F56124D3C1251595F4408FF2F
:1005600090FC16124D3C124F3390FC06124D3CF994
:10057000900025124F56124D3C1251605FFF90FCC7
:1005800016124D3C12505F90FC09124D3C1250FC6B
:10059000706812513E7063125144705E12509D702B
:1005A0005990FC06124D3C1250FC702612513E70C0
:1005B00021125144701C12509D7017900075124FFB
:1005C00056124D3CF990007512194BC39F502BE900
:1005D000800690FC09124D3C2436F9E43AFAC00337
:1005E000C002C00190FC06124D3C2436125094D03B
:1005F00001D002D0037F48124E4090FC06124D3CC1
:10060000125152FF90FC16124D3CF9121932FE6F36
:100610007021900001124F73124D3C125159B507D1
:100620001290FC16124D3C124F6F124D3C1251604D
:100630006F6003124E4590FC06124D3CF99000236A
:10064000EE1219AC90FC16124D3C900001124F7244
:10065000124D3CF9900024EF1219AC90FC16124D8B
:100660003C124F6F124D3CF9900025EF1219AC7EF1
:10067000007F1E7D0090FC16124D3C1251A37F2D71
:100680007D0090FC19124D3C1251A37F037D009018
:10069000FC1C124D3C1251A37F0C7D0090FC1F12DC
:1006A0004D3CF912224EE490FC12F090FC14F090B4
:1006B000FC13F090FC15F090FC06124D3C124F9884
:1006C000640160030208D090FC09124D3C124F985F
:1006D00060030208D0302F0302182090FC06124D50
:1006E0003CF990008312194BFF54C0440190FC1256
:1006F000F06F6003124E45125137705B124F9190AC
:10070000FC06124D3C124DAA506D124D7FFF54E075
:1007100064407031124DFA124F3B90FC11E0D3123D
:100720004DB2505390FC13E0C3941E501390FC063E
:10073000124D3C124D80FF90FC16124D3C124E5A49
:1007400012504680D590FC06124D3C124D74124D4D
:1007500087124DE10206FF90FC06124D3CF9900015
:100760008412194B541F64066003124E45124ECA80
:10077000124D3CF912A9DD124F9190FC06124D3C2E
:10078000124DAA504B124D7FFF54E06420702F127F
:100790004DFA124F3B124FAEFED39F503390FC14D4
:1007A000E0C3942D5012124CC3124DBA124F1112C5
:1007B0004D3C124F5E12510312516702079590FC97
:1007C00006124D3C124D74124D87124DE102077A0C
:1007D000124F9190FC06124D3C124DAA506C124DD6
:1007E0007FFF54E064807050124DFA90FC0F124D60
:1007F00069124F67124D8AFF90FC1C124D3CF9EFB5
:10080000124F2C124D3C124D74FF04F0E92F124D83
:100810008AFF90FC1C124D3C124F3390FC06124D87
:100820003C124D74FF04F0E92F124D8AFF90FC1C1E
:10083000124D3C12505F801290FC06124D3C124D3E
:1008400074124D87124DE10207D3124F9190FC06AE
:10085000124D3C124DAA504A124D7FFF54E0646085
:10086000702E124DFA124F3B124FAEFED39F50DD49
:10087000125114501690FC06124D3C124D80FF9000
:10088000FC1F124D3C90FC15124E5D12504680D854
:1008900090FC06124D3C124D74124D87124DE10230
:1008A000084D90FC06124D3C125195124D3CF97EBC
:1008B000007F8012190C90FC06124D3C12510B1255
:1008C0004E4590FD9FE06003021436D22F0214368D
:1008D00090FC09124D3C124F98640160030213F220
:1008E000124EB0124E89C39480EE648094805016EC
:1008F00090FC09124D3CF974801250D5124E6B7069
:10090000E2124EE980DD90FD9EE0604A90FC061206
:100910004D3C2400124FEC54FD124F2C124D3C1252
:10092000510B124E4590FC09124D3C124EBB124D1C
:100930003CF912A9DD124E1990FC19124D3C121807
:1009400026124D3CF912AF9D90FD9FE0600302140A
:1009500036D22F021436302F0302182090FC0612D4
:100960004D3C1250F530E129124FEA54FD12199A0C
:1009700090FC09124D3C1250E7C003C002C0019028
:10098000FC06124D3C125092D001D002D003124E00
:100990003E90FC09124D3CF9900083124F73124DAA
:1009A0003CF990008312194BFE5F54F0444190FCD7
:1009B00012F06E6003124E451251376003020A971F
:1009C000124F9190FC06124D3C124DAA5041124D0F
:1009D0007FFF54E064407025124DFA801B124FAE29
:1009E000FED39F50DE90FC06124D3C124D80FF90CE
:1009F000FC16124D3C124E5A12504680E090FC06F6
:100A0000124D3C124D74124D87124DE10209C31272
:100A1000506790FC09124D3C124E4CC39F4003029C
:100A20000BA7124E796440705C90FC10124E0212BB
:100A30004FFD12516F50DBE4124EB4124DCA5024D8
:100A4000124DEC124D3C124DBA547FFF90FC161221
:100A50004D3C124DC2547F6F600A124E7270DC1210
:100A60004EE980D7124EF04016124DEC124D3C125A
:100A70004DBAFF90FC16124D3C124E5A124E4512C2
:100A8000517B020A32124DEC124D3C124DBA90FCD1
:100A90000E124DE4020A12124F9190FC06124D3CC8
:100AA000124DAA4003020BA7124D7F54E064406030
:100AB00003020B9512506790FC09124D3C124E4CEC
:100AC000C39F4003020BA7124E7964406003020BE0
:100AD00086124F7B90FC06124D3C124D74124F064D
:100AE000124FF4A3E004F090FC0EE0FF90FDA0E4B0
:100AF000F0A3EFF0124FAED39F4003020BA790FD7F
:100B0000A0A3E090FC0EF090FC10E0124E53D39F97
:100B1000504190FC06124D3C124D74124F0712507A
:100B200004124D3C124DC2FE547F6F702090FC1396
:100B3000E0C3941E501790FC06124D3C124D7412E7
:100B40004F074EFF90FC16124D3C124E5A124FFDAD
:100B5000020B0790FC13E0FF602390FC06124D3C53
:100B6000124D74124F07FEEF24FFFDEC34FFFC9092
:100B7000FC16124D3C124DC26E60058000124E45AF
:100B8000125046020AF4124DEC124D3C124DBA12AC
:100B90004F86020AB790FC06124D3C124D74124D5E
:100BA00087124DE1020A9A90FD9FE0FF6401600800
:100BB000EF64036003020E91124F9190FC06124DF8
:100BC0003C124DAA5042124D7FFF54E06420702623
:100BD000124DFA125046124FAEFED39F50DD124C0A
:100BE000C3124DBA124F11124D3C124F5E125103F7
:100BF000125167020BD690FC06124D3C124D741236
:100C00004D87124DE1020BBB12506790FC09124D4B
:100C10003C124E4CC39F4003020DCA124E79642011
:100C20006003020DBB124F7B124FFD12516F50DB60
:100C3000E4124EB490FC14124DCD4003020D5F122D
:100C40004DEC124D3C124DBA5478FF90FC19124DE8
:100C50003C124DC2FE54786F6003020D5290FC0EA0
:100C6000E0124EDF124D3C124DC25407FFEE540706
:100C7000FED39F4004AF06800090FC0EE0124EDFD2
:100C8000124D3C124DC254784FFF90FC19124D3C4E
:100C9000F990FDA0E0FCA3E0FDF5828C83EF121932
:100CA000AC90FC0EE02481124DF2124D3C124DBA74
:100CB000FF90FC19124D3CF9ED2401FDE43C12516A
:100CC0004A4F8D828C831219AC124E89F5828E8325
:100CD00012194B5478FDBD013690FC19124D3CF9A8
:100CE000EF2402FFE43EFEE92FF9EA3EFAC003C01A
:100CF00002C0011219321250CD124EE1124D3C12B7
:100D00004DC24FD001D002D00312199A020D5F904C
:100D1000FC0EE090FC09124D36124DBAFF90FC1902
:100D2000124D3CF990FDA1E02402FD124FE3125157
:100D30004AFED39F4004AF06800D1250CE124DF2F2
:100D4000124D3C124DBAFF90FC19124D3C124F5EF1
:100D5000800D90FDA1E02403124FE2F0020C3490CC
:100D6000FC14124EF3404E12511C90FC09124D3CE3
:100D7000124DC2FD90FC19124D3C1250A6ED1219F5
:100D8000AC125183124D3C124DBAFF90FC14E0247A
:100D900001124F18124D3C124F5E1250CE124DF2FE
:100DA000124D3C124DBA124F11124D3C124F5E12B1
:100DB0005103124E4512517B020C2B124DEC124D79
:100DC0003C124DBA124F86020C0B124F9190FC064A
:100DD000124D3C124DAA40030210D6124D7F54E032
:100DE00064806003020E7F12506790FC09124D3C34
:100DF000124E4CC39F40030210D6124E796480708D
:100E00006F124F7B90FC06124D3C124D44124F67FF
:100E1000124D8A124E5304F0125007124D3C124DDF
:100E2000C24FFF90FC1C124D3CF9EF124F2C124D9B
:100E30003C124D74124F67124D8A124E53124EDC03
:100E4000124D3C124DC24FFF90FC1C124D3C124FF4
:100E50003390FC06124D3C124D74124F67124D8AAE
:100E6000124E53124EDC124D3C124DC24F0210A9CD
:100E7000124DEC124D3C124DBA124F86020DEA9003
:100E8000FC06124D3C124D74124D87124DE1020DBD
:100E9000CD124F9190FC06124D3C124DAA40030218
:100EA0001006124D7FFF54E064206003020FF4121D
:100EB0004DFA125046124FAED39F50D81250679041
:100EC000FC09124D3C124E4CC39F4003020FEE1220
:100ED0004E7964206003020FDF124F7B124FFD90AA
:100EE000FC10E0124E53D39F50D590FC06124D3C9F
:100EF000124D74124F07125004124D3C124DC25441
:100F00007F6F6003020FA890FC14E0C3942D400390
:100F1000020FA812511C124DC3FD90FC19124D3C3A
:100F20001250A6ED1219AC90FC0FE02481FDE433C1
:100F3000FC90FC06124D3C124DC2FD125183124D25
:100F40003C124DBA5DFF90FC14E0FE2401124F18D4
:100F5000124D3C124F5E8E8275830012194B5478ED
:100F600064017016124D2F124DBA1250CD124EE17F
:100F7000124D3C124DC25FFF8022124D2F124DBA0E
:100F80001250CD124EE1124D3C124DC2FEC39F5085
:100F900004AF068007124D2F124DBAFF124F1212E6
:100FA0004D3C124F5E12510390FC14E0FF602790FD
:100FB000FC06124D3C124D74124F07547FFEEF2475
:100FC000FDFDEC34FFFC90FC19124D3C124DC25457
:100FD0007F6E60058000124E4512517B020EDF12BB
:100FE0004DEC124D3C124DBA124F86020EBF1251FB
:100FF00067020EB590FC06124D3C124D74124D87DF
:10100000124DE1020E94124F9190FC06124D3C12CB
:101010004DAA40030210D6124D7F54E06480600355
:101020000210C412506790FC09124D3C124E4CC382
:101030009F40030210D6124E7964807078124F7B65
:1010400090FC06124D3C124D44124F67124D8A120D
:101050004E5304F0125007124D3C124DC25FFF90E8
:10106000FC1C124D3CF9EF124F2C124D3C124D74EA
:10107000124F67124D8A124E53124EDC124D3C1223
:101080004DC25FFF90FC1C124D3C124F3390FC068A
:10109000124D3C124D74124F67124D8A124E53126C
:1010A0004EDC124D3C124DC25FFF90FC1C124D3CB9
:1010B00012505F8021124DEC124D3C124DBA124F6E
:1010C0008602102690FC06124D3C124D74124D877C
:1010D000124DE1021009124F9190FC06124D3C1284
:1010E0004DAA4003021436124D7F54E06460600341
:1010F0000213E012506790FC09124D3C124E4CC393
:101100009F4003021436124E79646060030213D1CB
:10111000124F7B90FC06124D3C124D74124F06127A
:101120004FF4A3E004F01251376003021234A3F02D
:10113000A3F0124FB84008125012400302133E9021
:10114000FC15E0C3940C4003021229124E89640678
:101150004E6018EF64084E6012EF64094E600CEFA9
:10116000640A4E6006EF640B4E703790FC06124D19
:101170003C124D74124D91124E92124D3C124DC2C2
:10118000FEEFD39E400F90FC06124D3C124D7412A0
:101190004D910211F812502C124D3C124DBAFF0223
:1011A00011F8124E891250B1503790FC0CE030E12A
:1011B000221250BA124D3C124DBAFF90FC1F124D34
:1011C0003C90FC151250A912194B6F6003124E454A
:1011D0000211F890FC06124D3C124D74124D918094
:1011E0001790FC06124D3C124D74124D91124E9206
:1011F000124D3C124DC24FFF90FC1F124D3CF99016
:10120000FC15124E5E124E891250B1401C90FC0625
:10121000124D3C124D7412504DFD90FC1F124D3C6E
:10122000124DBA6D6003124E45124E727003124E8B
:10123000E9021132E4124EB4124FB8400302133ED9
:10124000125012400302133E90FC15E0C3940C4070
:1012500003021333124E8964064E6018EF64084E81
:101260006012EF64094E600CEF640A4E6006EF6492
:101270000B4E703790FC06124D3C124D74124D917E
:10128000124E92124D3C124DC2FEEFC39E500F9073
:10129000FC06124D3C124D74124D91021302125075
:1012A0002C124D3C124DBAFF021302124E891250FD
:1012B000B1503890FC0CE030E1231250BA124D3C92
:1012C000124DBAFF90FC1F124D3CF990FC151250C4
:1012D000AA12194B6F6003124E4502130290FC06CE
:1012E000124D3C124D74124D91801790FC06124D18
:1012F0003C124D74124D91124E92124D3C124DC241
:101300005FFF90FC1F124D3CF990FC15124E5E12CF
:101310004E891250B1401C90FC06124D3C124D7487
:1013200012504DFD90FC1F124D3C124DBA6D6003E2
:10133000124E45124E727003124EE902123890FCA2
:101340001F124D3CF9740312519C124D3CF9124F7F
:101350009F90FC0CE030E20A90FC1F124D3CF91209
:10136000508312511450037405F090FC15E0FFC334
:101370009407402F90FC1F124D3C2405F9E43AFAE3
:1013800012193254BF12519C124D3CF990000612B2
:10139000194BFEC3942D500280027E2D900006EE64
:1013A0001219AC90FC0FE0247FFDE433FC90FC06A6
:1013B000124D3C124DC2541F6F6003124E4590FCFB
:1013C00011E00490FC0FF0A3E00490FC0EF0021476
:1013D00036124DEC124D3C124DBA124F860210F6E9
:1013E00090FC06124D3C124D74124D87124DE102D5
:1013F00010D990FC06124D3C2400124FEC54FD1203
:101400004F2C124D3C12510B124E4590FC09124DBF
:101410003C124EBB124D3CF912A9DD124E1990FC44
:1014200019124D3C121826124D3CF912AF9D90FD39
:101430009FE07002D22F90FC06124D3C124F986430
:101440000160030217AD90FC13E0C39401500A122F
:101450004ECA124D3CF912A9DD90FD9FE0B4042A5A
:1014600090FC917401F0A374FCF0A37414F090FC50
:101470001CE0F9A3E0FAA3E090FC94124E3490FC37
:1014800019124D3CF912A564801690FC14E0C39427
:1014900003500D124E1990FC19124D3CF912A83947
:1014A000125114501890FD227401F0A374FCF0A3A3
:1014B0007415F090FC1F124D3CF912AF9D90FC0C7E
:1014C000E020E009D312511540037405F0E4124EF8
:1014D000B4124DCA501690FC16124D3C124DC2204B
:1014E000E70A124E7270EA124EE980E5124EF040A1
:1014F0000F90FC16124D3CF9121932448012199AC1
:10150000E490FC0FF090FC06124D3C124D74124F0B
:1015100067F9EE3AFA7402124F2C124D3C124D74D8
:10152000FF04F0E92FF9EE3AFA740312199A90FCCD
:1015300013E0240BFFA3E02FFFA3E02FFF90FC0696
:10154000124D3C124D74124E0E90FC14E075F01EBC
:101550008412197812504690FC12E0FF90FC06129B
:101560004D3C124D74FE04F0EE124E1090FC13E050
:101570004440FF90FC06124D3C124D74FE04F0EE08
:10158000124E10E4124EB4124DCA502090FC1612A6
:101590004D3C124DC2FF90FC06124D3C124D741290
:1015A0004E0A124E7270E0124EE980DB90FC14E09D
:1015B000C3941E500302163790FC06124D3C124D88
:1015C00074124F67F9EE3AFA743E12199AE4124E09
:1015D000B4124E89C3941EEE64809480502090FC17
:1015E00019124D3C124DBAFF90FC06124D3C124DA3
:1015F00074124E0A124E7270D8124EE980D390FCCB
:1016000014E024E2FFE434FFFE90FC19124D3C2468
:101610001EF9E43AFAC003C00290FC19A3E0FAA351
:10162000E0F8AC02AD03D002D00312190C90FC1408
:10163000E024E2F00215AC90FC14E04420FF90FCA2
:1016400006124D3C124D74124E0AE4124EB490FC38
:1016500014124DCD502090FC19124D3C124DC2FF7A
:1016600090FC06124D3C124D74124E0A124E7270CE
:10167000DD124EE980D890FC06124D3C124D7412DA
:101680004F67F9EE3AFA748312199A90FC1C124DC6
:101690003CF9121932FF90FC06124D3C124D7412A7
:1016A0004E0A90FC1C124D3CF9900001124F73122F
:1016B0004D3C124D74FE04F0EE124E1090FC1C12C4
:1016C0004D3C124F6F124D3C124D74FE04F0EE1261
:1016D0004E1090FC15E04460FF90FC06124D3C1249
:1016E0004D74FE04F0EE124E10E4124EB490FC1550
:1016F000124DCD502090FC1F124D3C124DC2FF9058
:10170000FC06124D3C124D74124E0A124E7270DDE0
:10171000124EE980D8E4124EB4124DCA506290FCC9
:101720000FE0C3946E505990FC16124D3C124DC2FE
:10173000547FFF6401603EEFC3943C5038EF75F076
:1017400012A42438F9744235F0FA7BFFC003C002BA
:10175000C00190FC06124D3C124D747E0029F9EE3A
:10176000125096D001D002D0037F1212190C90FCB7
:101770000FE02412F0124E727003124EE902171994
:1017800090FC0FE0FFFDC374809DFDE49400FCC05D
:1017900004C00590FC06124D3C1250E7EF7C002976
:1017A000F9EC3AFA7D00D007D00612224E124EAF65
:1017B000124E8912507A501390FC06124D3C124D75
:1017C000BA124E6B70EA124EE980E51250DF90FCBF
:1017D00006124D3CF990007FEF1219AC124F99643C
:1017E00001703D90FC06124D3CF99000FEE4124E53
:1017F000AC124E8912507A501690FC06124D3C12D3
:1018000050E7124D9F124E6C70E7124EE980E212C3
:1018100050DF90FC06124D3CF99000FFEF1219AC1E
:1018200090FC0DE0FF22F912A83990FD227401F01E
:0C183000A374FCF0A37415F090FC1F22C0
:102D9D0049646C65005472616E736D69745F4D6545
:102DAD007373616765005365745F4C6F6769636129
:102DBD006C5F4164647265737300436F6E6E65631F
:102DCD007400446973636F6E6E6563740053746150
:102DDD006E646279005374616E6462795F416C6CEC
:102DED00005265636F72645F43757272656E740035
:102DFD005265636F72645F43757272656E745F4F77
:102E0D006666005365745F54696D65725F50726FCD
:102E1D006772616D00436C6561725F54696D6572B7
:102E2D005F50726F6772616D004765745F4D656EBF
:102E3D00755F4C616E677561676500416E6E6F758C
:102E4D006E63655F4D656E755F4C616E677561672D
:102E5D006500436F6E74726F6C5F4465636B0053F6
:102E6D00656C6563745F54756E65725F53657276DC
:102E7D0069636500436F6E74726F6C5F54756E6538
:102E8D00720053656E645F56656E646F725F436F5B
:102E9D006D6D616E640042726F6164636173745F26
:102EAD0056656E646F725F436F6D6D616E64005633
:102EBD00656E646F725F52656D6F74655F42757498
:102ECD00746F6E5F507265737365640056656E64E2
:102EDD006F725F52656D6F74655F427574746F6E5E
:102EED005F52656C656173656400526571756573DC
:102EFD00745F4D656E7500557365725F436F6E74CB
:102F0D00726F6C5F50726573736564005573657293
:102F1D005F436F6E74726F6C5F52656C6561736544
:102F2D006400526571756573745F53797374656D63
:102F3D005F417564696F5F4D6F64650055706461C5
:102F4D0074655F4465766963655F496E666F0052AF
:102F5D006571756573745F496D6167655F56696508
:102F6D00775F4F6E00526571756573745F54657848
:102F7D00745F566965775F4F6E00416E6E6F756E4B
:102F8D0063655F4163746976655F536F75726365E1
:102F9D00005365745F496E6163746976655F536F45
:102FAD007572636500526571756573745F446973FD
:102FBD00706C61795F4F53445F537472696E670033
:102FCD00496E666F726D5F4D656E755F537461749A
:102FDD007573005365745F53797374656D5F4175D7
:102FED0064696F5F4D6F6465005265706F72745FD9
:102FFD005265636F72645F537461747573005265CB
:10300D00706F72745F54696D65725F53746174751E
:10301D0073005265706F72745F54696D65725F43B2
:10302D006C65617265645F53746174757300556E80
:10303D00737570706F727465645F4D6573736167DE
:10304D006500496D6167655F566965775F4F6E0015
:10305D00546578745F566965775F4F6E0041637490
:10306D006976655F536F7572636500496E61637450
:10307D006976655F536F757263650052657175652D
:10308D00737465645F666F725F5374616E646279A9
:10309D0000496E666F726D65645F4D656E755F4C50
:1030AD00616E677561676500526563656976656414
:1030BD005F56656E646F725F436F6D6D616E640018
:1030CD0052656365697665645F56656E646F725FA0
:1030DD0052656D6F74655F427574746F6E5F50727B
:1030ED0065737365640052656365697665645F56E3
:1030FD00656E646F725F52656D6F74655F42757456
:10310D00746F6E5F52656C656173656400446973BD
:10311D00706C61795F4F53445F537472696E6700D1
:10312D00496E666F726D65645F4D656E755F537444
:10313D00617475730052656365697665645F557377
:10314D0065725F436F6E74726F6C5F5072657373EF
:10315D0065640052656365697665645F5573657274
:10316D005F436F6E74726F6C5F52656C65617365F2
:10317D00640053797374656D5F417564696F5F4D5C
:10318D006F64655F536574004465766963655F4977
:10319D006E666F5F4368616E676564005365745F4B
:1031AD0053747265616D5F5061746800526571751D
:1031BD0065737465645F5265636F72645F437572A6
:1031CD0072656E74005265717565737465645F52D6
:1031DD0065636F72645F43757272656E745F4F667F
:1031ED0066005265717565737465645F5365745FD0
:1031FD0054696D65725F50726F6772616D005265D3
:10320D00717565737465645F5365745F54696D653D
:10321D00725F50726F6772616D5F5469746C650097
:10322D005265717565737465645F436C6561725F3A
:10323D0054696D65725F50726F6772616D00526592
:10324D00717565737465645F666F725F4D656E75DC
:10325D00005265717565737465645F436F6E74724A
:10326D006F6C5F4465636B0053656C656374656477
:10327D005F54756E65725F53657276696365005252
:10328D0065717565737465645F436F6E74726F6C91
:10329D005F54756E65720052657175657374656402
:1032AD005F666F725F53797374656D5F41756469A5
:1032BD006F5F4D6F646500526F7574696E675F4F18
:1032CD00666600443D307825302E325820446565C1
:1032DD007020436F6C6F7220446574656374656410
:1032ED000D0A00443D307825302E32582034204FC1
:1032FD00757470757420537570706F72740D0A004B
:10330D00443D307825302E32582054782054524583
:10331D0047203D20307825302E32580D0A00455279
:10332D00524F523A204E3D307825302E32582041A2
:10333D004B535620524459202D204D435520494979
:10334D00432025640D0A004552524F523A204E3DFE
:10335D00307825302E325820414B535620726561FE
:10336D0064202D204D4355204949432025640D0AE5
:10337D00004552524F523A204E3D307825302E3274
:10338D005820414B53562072656164202D204B65AA
:10339D00792057726F6E670D0A004552524F523A9F
:1033AD00204E3D307825302E3258205478205269E9
:1033BD002072656164202D204D43552049494320DD
:1033CD0025640D0A004552524F523A204E3D307839
:1033DD0025302E325820424B5356207265616420A1
:1033ED002D20444E204444432025640D0A004552AF
:1033FD00524F523A204E3D307825302E32582042D1
:10340D004B53562072656164202D204B65792057F2
:10341D00726F6E670D0A004552524F523A204E3D63
:10342D00307825302E32582052782052692072651E
:10343D006164202D20444E204444432025640D0A10
:10344D00004552524F523A204E3D307825302E32A3
:10345D0058204B5356204649464F207265616420D3
:10346D002D20444E204444432025640D0A0045522E
:10347D00524F523A204E3D307825302E3258204B47
:10348D005356204649464F2072656164202D204BCE
:10349D0065792057726F6E670D0A004552524F5273
:1034AD003A204E3D307825302E325820454449443F
:1034BD002062302072656164202D20444E204444EA
:1034CD00432025640D0A004552524F523A204E3D7D
:1034DD00307825302E3258204544494420436865C4
:1034ED00636B206661696C65642C207045444944AA
:1034FD005B3132365D3D307825302E3258203E20FE
:10350D00380D0A004552524F523A204E3D30782523
:10351D00302E32582045444944206269207265613D
:10352D0064202D20444E204444432025640D0A0080
:10353D004552524F523A204E3D307825302E32585A
:10354D00204544494420636865636B73756D206540
:10355D0072726F720D0A005741524E494E473A2012
:10356D00443D307825302E3258204E6F2045504343
:10357D00432064657465637465640A0D00443D30D1
:10358D007825302E325820455043432064657465AC
:10359D0063746564205665723D25642E25640A0D9D
:1035AD00005741524E494E473A204E6F20446576A2
:1035BD0069636520666F756E640D0A005741524E42
:1035CD00494E473A204E6F20417564696F205379FB
:1035DD007374656D20666F756E640D0A00574152E8
:1035ED004E494E473A20443D307825302E325820F2
:1035FD0045504343204576656E74204D697373695C
:10360D006E670D0A004552524F523A20443D3078B4
:10361D0025302E3258204550434320436F6D6D6148
:10362D006E642054696D652D6F75740D0A004552D9
:10363D00524F523A20494943206661696C656420B6
:10364D0025642C20494943416464723D307825300E
:10365D002E32582C20526567416464723D307825B6
:10366D00302E32580D0A00FF2D9DFF2DA2FF2DB3D8
:10367D00FF2DC7FF2DCFFF2DDAFF2DE2FF2DEEFF22
:10368D002DFDFF2E10FF2E22FF2E36FF2E48FF2E72
:10369D005FFF2E6CFF2E81FF2E8FFF2EA3FF2EBC02
:1036AD00FF2ED9FF2EF7FF2F04FF2F19FF2F2FFF0E
:1036BD002F49FF2F5CFF2F72FF2F87FF2F9EFF2FAC
:1036CD00B2FF2FCDFF2FE0FF2FF6FF300BFF301F86
:1036DD00FF303BFF304FFF305DFF306AFF3078FF2A
:1036ED003088FF309EFF30B5FF30CDFF30F3FF3116
:1036FD001AFF312DFF3142FF3160FF317FFF3195D0
:10370D00FF31A9FF31B9FF31D2FF31EFFF320BFF8E
:10371D00322DFF324BFF325EFF3275FF328CFF329E
:04372D00A4FF32C4FF
:0C8C7A0001680042FC4800000264000099
:106D670090FC97E0FBA3E0FAA3E0F9121932FF9039
:106D7700FC9AE0FBA3E0FAA3E022F090FC4EE47556
:106D8700F001121A81FE748025F0F58274FF3EF53A
:106D9700837469F090FC4EE475F001121A81FE7459
:106DA7008025F0F58274FF3EF58322F9121932042B
:106DB700FF90FD097B00E47A007922F0A304F0221A
:106DC700F0A3EDF0A3EBF0A3EAF0A3E9F022121988
:106DD7003204FF90FCC87B00E47A007922F0A322FA
:106DE700F9121932FF90FB39E4F0A3EFF02290FF7C
:106DF70080F090FC5AE47B017AFF7980F0A322F9B6
:106E070090000102194B2407F9E43AFA90FCC8E410
:106E1700F0A322F9121932FF90FD88E4F0A30422AF
:106E27007B007A00792290FC5AE4F0A322F9121928
:106E370032FFE490FD88F0A32290FC4AE090FB3BF0
:106E4700FFE4F0A3EFF022F990FC4EE0FEA3E0F59B
:106E5700828E8302194BF990000212194BFF9000A2
:106E67000312194BFD22F9121932FF7B017AFF79C0
:106E770080227967E7C4F8540FC868FF19E7C4543C
:106E8700F048FEE42FFDEE22F9A3E0FFA3E090FC1B
:106E97005ACFF0A3EFF0222FF9EA3EFA900004123E
:106EA700194BFF90000512194BFD2290FC4AEFF099
:106EB700E0FE2204F0A3F07D74FF22F990FD09E4BF
:106EC700F0A3222401F9E43AFA021932E490FC4EC5
:106ED700F0A3F0227405F0E4A3F07D757F0122F999
:106EE70012193204FF2290FCB2E0FD90FB39E4F066
:106EF700A3EDF0A32290FC4EE0FDA3E090FCC8CDEB
:106F0700F0A3EDF022A3E4F0A3E522F07BFF7A33B0
:106F1700790D2290FC4EE4F0740AA3F0E4A3F0A3E9
:106F2700F02290FC4FE004F02290FC4EE004F022A7
:106F370090FD42E014FF90FD41E02290FC4EE0FE00
:106F4700A3E0FFC39406EE6480948022D390FC4FA5
:106F5700E0940090FC4EE064802290FC51E004F045
:106F67002290FC50E004F022C390FC51E09403907F
:106F7700FC50E064809480227480F0E4A3F07DA14B
:106F87007F012290FC4AE0FF90FB3B22E025E0FFD7
:106F970090FC4EE033FE90FC5222C390FDC5E09476
:106FA700E890FDC4E0940322A3E024FDF090FC4E9A
:106FB700E034FFF02204F0A3F07DA0FF2290FD87CC
:106FC700E0FF7401A8070822E52225E0F52222F058
:096FD700A37402F07D747F012215
:10863E0090FC4B126DCC90FD28E0F9A3E0FAA3E07C
:10864E0090FC52C9126DCD90FC52126D79126E5D76
:10865E0012777C90FC52126D79126E5D7B0212675E
:10866E00D290FC52126D79F9121932FF126E07FD7B
:10867E001278E390FC52126D79F9121932FF126ED4
:10868E0007FD7B011267D212AA0D7D087F061277B5
:10869E007C7B017D087F061267D2126ED3126F4269
:1086AE00501FEF25E0FFEE33FE90FC52126D791253
:1086BE006E9E7B011267D2126F297003126F30808B
:1086CE00DCE4FB7D01FF12A8A57B02E4FD7F011215
:1086DE00A8A57BFF7A9E7994E4FF12B0A390FDC902
:1086EE0074FEF07BA0E4FD12A6DF7BFF7A00794ECC
:0A86FE00E4FF12B0927D0102A626EF
:10AA0D0090FC52126D79F9121932FF126E07FD1278
:10AA1D0078E312940490FC52126D79F9121932FFF9
:0CAA2D00126E07FD12777C7F0402B1243A
:10B0470090FC52126D79126E5D12777C7D02E4FFDF
:03B0570002AD2027
:10B08000E4FDFF12AD2090FC52126D79126E5D024C
:02B0900078E363
:1090F90090FDE2126DCC90FDE2126D79F9ED121935
:109109009A90FDE2126D79F9900001E41219AC12FE
:109119006DB37D0512870890FC4AE07024E5226052
:109129002090FDE2126D79126DE77BFF7A3279D0DA
:1091390012A3B190FDE2126D79126ECA4440121960
:109149009A75220890FDE2126D79F9121932126DA1
:10915900B77D0712870890FDE2126D79126DB27D15
:109169000712870890FC4AE0702330132090FDE233
:10917900126D79126DE77BFF7A3279F012A3B19003
:0E918900FDE2126D79126ECA448012199A220C
:0DB0FE00126E0730E6047F0180027F002201
:1096500090FDE5126DCC90FDE5126D79126E06302D
:10966000E51F30E60820E74C126E1B802690FDE5D2
:10967000126D79126E1A1296D1126D79126E1A80CD
:109680002B90FDE5126D79126E0630E60D20E72471
:10969000126E35F07B067D06801790FDE5126D7920
:1096A000126E341296D1126D79126E34F07B047DF5
:1096B0000A12A4DB90FDE5126D79126DB27D0612DF
:1096C000870890FDE5126D79126DE7126F0C02A309
:0D96D000B1F07B057D0A12A4DB90FDE522C0
:10AABD0090FDE8126DCCED90FDE8600A126D7912F3
:10AACD006ECA44208008126D79126ECA54DF1219B5
:0BAADD009A90FDE8126D79F902965086
:10A3160090FDEB126DCC90FDEB126D79126E06304E
:10A32600E40830E61C126E35800F90FDEB126D7955
:10A33600126E0630E60B126E1BF07B077D0612A42A
:10A34600DB90FDEB126D79126DB27D0612870890D7
:0EA35600FDEB126D79126DE7126F0C02A3B1D0
:10AAE80090FDEE126DCCED90FDEE600A126D7912BC
:10AAF8006ECA44108008126D79126ECA54EF12198A
:0BAB08009A90FDEE126D79F902A31681
:10A7570090FDF1126DCC90FDF1126D79126E0630FD
:10A76700E60B126E1BF07B057D0612A4DB90FDF154
:10A77700126D79126DB27D0612870890FDF1126D88
:0AA7870079126DE7126F0C02A3B106
:10AA390090FDF4126DCC90FDF4126D79126E063012
:10AA4900E708126E35F07B03800C90FDF4126D79E6
:0CAA5900126E34F07B017D0712A4DB229A
:109A8D0090FDF7126DCC90FDF7126D79126E0630C8
:109A9D00E634752208121932126DB77D051287084A
:109AAD0090FDF7126D79126E0630E7057522C280B2
:109ABD000A75229690FDF7126D79F9121932126D11
:109ACD00B77D0612870890FDF7126D79F912965041
:109ADD0090FDF7126D79F912A31690FDF7126D79BD
:109AED00126E0630E708126E1BF07B03800B90FDA3
:0F9AFD00F7126D79126E1AF0FB7D0712A4DB22AF
:10A97A0090FDFA126DCC90FDFA126D79126DB27DCE
:10A98A000712870890FDFA126D79126E0630E708F1
:10A99A00A216821782138006A21682178211E43346
:02A9AA00FF228A
:0EB0D400126DB37D07128708A215E433FF2228
:09B18A0090FDFD126DCC7F002246
:0EB0E200126DB37D08128708A216E433FF2218
:0EB0F000126DB37D40128708A210E433FF22D8
:10000E00121932FF90FD2E126D79126EC27403F02A
:05001E007D500287087F
:10AF3D00121932FF90FCDD126D79F9A3E0FD126E4E
:08AF4D00C3EDF07D80028708CE
:10AFCB0012193204FF90FD34126D79126EC274089F
:06AFDB00F07D4102870831
:10005600121932FF90FD3A126D79126EC27414F0C5
:050066007D6002870827
:10AE4E0090FE00126DCC90FE00126D79F912A12ABF
:10AE5E0090FE00126D79126E34F0FB7D0802A4DBB9
:10AD670090FE03126DCC90FE03126D79F912A12AA1
:10AD770090FE03126D79126E1AF0E4FB7D0802A4AF
:01AD8700DBF0
:10AD880090FE06126DCC90FE06126D79F912A12A7A
:10AD980090FE06126D79126E1AF07B077D0802A4E8
:01ADA800DBCF
:10ADA90090FE09126DCC90FE09126D79F912A12A53
:10ADB90090FE09126D79126E34F07B077D0802A4AA
:01ADC900DBAE
:10ADCA0090FE0C126DCC90FE0C126D79F912A12A2C
:10ADDA0090FE0C126D79126E1AF0E4FB7D0F02A43C
:01ADEA00DB8D
:10AE6E0090FE0F126DCC90FE0F126D79F912A12A81
:10AE7E0090FE0F126D79126E34F0FB7D0F02A4DB83
:109CF20090FDA2126DCCA3EDF012A12A90FDA2124A
:109D02006D79126DB27D091287083011037F01222D
:109D120090FDA5E0FF12A1D2E4F522FB90FC5A12BD
:109D22006DBEA3F07D60FF1275D1E4F522FB90FCBD
:109D32005A126DE0126FBC1275D1126EB2C006904B
:109D4200FC5A126DBB126F821275D1D0E04F90FC9B
:0A9D52004AF070037F02227F002216
:1000260090FE12126DCC90FE12126D79F912A12A71
:1000360090FE12126D79126DB27D09128708A21216
:04004600E433FF227E
:10ADEB0090FE15126DCC90FE15126D79F912A12AF9
:10ADFB0090FE15126D79126E1AF0E4FB7D0E02A413
:01AE0B00DB6B
:10AE8E0090FE18126DCC90FE18126D79F912A12A4F
:10AE9E0090FE18126D79126E34F0FB7D0E02A4DB5B
:10AE0C0090FE1B126DCC90FE1B126D79F912A12ACB
:10AE1C0090FE1B126D79126E1AF07B047D0F02A44A
:01AE2C00DB4A
:10AE2D0090FE1E126DCC90FE1E126D79F912A12AA4
:10AE3D0090FE1E126D79126E34F07B047D0F02A40C
:01AE4D00DB29
:10AA650090FCE1126DCC90FCE1126D79F912A12AEE
:10AA750090FCE1126D79F9121932FF90FCE5126D27
:0CAA850079126EC27408F07D150287087B
:10A6650090FDA6126DCCA3EDF012A12A90FDA612C5
:10A675006D79126DB27D0F12870890FC4AEFF0607C
:10A68500167BFF7A33792B90FDA9E0126DEB126EE4
:0DA695004012A3B17F0022A217E433FF2280
:108E720090FCE8126DCCA3EDF012A12A90FCE8124E
:108E82006D79126EE690FCEC126D79126EC2740767
:108E9200F07D1D12870890FC4AEFF060127BFF7A8A
:108EA20033795490FCEBE0126DEB126F8A8058120A
:108EB2006ED3A3F0A3F0F522752201E522601A9089
:108EC200FCEC126D79126E4E55226008126F6170C1
:108ED20003126F68126FCF80E2126F297003126F54
:108EE2003090FC4EE07004A3E0640570CB90FC501F
:108EF200E07004A3E0641460197BFF7A33797E90FA
:108F0200FCEBE0FF90FB39E4F0A3EFF012A3B17F9A
:058F120000227F012296
:10AA910090FCEF126DCC90FCEF126D79F912A12AA6
:10AAA10090FCEF126D79F9121932FF90FCF3126DDF
:0CAAB10079126EC27405F07D1002870857
:10AB3E0090FE21126DCC90FE21126D79F912A12A90
:10AB4E0090FE21126D79126DB27D0F128708E522EB
:0AAB5E0030E1047F0180027F002235
:10A4950090FCF6126DCCA3EDF012A12A90FCF612F9
:10A4A5006D79126EE690FCFA126D79126EC2740225
:10A4B500F07D2212870890FC4AEFF060167BFF7A48
:10A4C5003379A790FCF9E0126DEB126E4012A3B13F
:06A4D5007F00227F01223E
:10AB680090FCFD126DCC90FCFD126D79F912A12AB2
:10AB780090FCFD126D79126EE690FD01126D79124E
:0AAB88006EC27408F07D25028708F4
:108BAB0090FDAB126DCC90FDAAEFF012A1D290FD0F
:108BBB00AB126D79F9E412199A90FDAB126D79F93C
:108BCB00126E2D126EBA1275D1126EB2C00690FDD6
:108BDB00AB126D79F9126E2D126EDB1275D1D0E0DE
:108BEB004F90FC4AF060127BFF7A3379D290FDAA4A
:108BFB00E0126DEB126F8A8056126ED3A3F0A3F0C6
:108C0B00752201E522601A90FDAB126D79126E4E42
:108C1B0055226008126F617003126F68126FCF805C
:108C2B00E2126F297003126F3090FC4EE07004A3B8
:108C3B00E0640570CB90FC50E07004A3E06414601A
:108C4B00197BFF7A3379FB90FDAAE0FF90FB39E4A7
:0D8C5B00F0A3EFF012A3B17F00227F0122F1
:10AEAE0012A1D275224090FC5A126DDD126EBA12AA
:0FAEBE0075D1126E2704126EDD1275D1AF2222EC
:10ABE60090FE5DEDF012A1D2752215126E27126E3F
:10ABF600BA1275D17B017AFE795D126E2D04F0A32F
:09AC060004F07D747F010275D198
:1001D90090FE24126DCC12A1D2752218126E27122C
:1001E9006EBA1275D190FE24126D79F9126E2D74C2
:0701F90008126FD60275D158
:10AC380090FE27126DCC12A1D2752210126E271227
:10AC48006EBA1275D190FE27126D79F9126E2D74B5
:07AC580005126FD60275D151
:109EFA0090FDAF126DCC90FDAEEFF012A1D290FDA5
:109F0A00AF126D79F9740812199A90FDAF126D7932
:109F1A00F9126E2D126EBA1275D1126EB2C0069077
:109F2A00FDAF126D79F9126E2D7402126EDD127583
:109F3A00D1D0E04F90FC4AF060167BFF7A34792446
:109F4A0090FDAEE0126DEB126E4012A3B17F0022BB
:039F5A007F012262
:10A7CB0090FE2A126DCC12A1D290FE2A126D79F94D
:10A7DB00744112199A90FE2A126D79F9126E2D128C
:10A7EB006EBA1275D190FE2A126D79F9126E2D7414
:07A7FB0002126EDD0275D1B0
:10A8020090FE2D126DCC12A1D290FE2D126D79F90F
:10A81200742012199A90FE2D126D79F9126E2D1272
:10A822006EBA1275D190FE2D126D79F9126E2D74D9
:07A8320014126EDD0275D166
:107E410090FD3E126DCC90FD3DEFF012A1D290FD60
:107E510041E0703B752243FB7A00792290FC5AF095
:107E6100A3126EBA1275D1126F3790FD3EB5070C91
:107E7100126D79F9126E2D126EDB803D126D79F95A
:107E8100126E2D7405F0A37401F07D75FF802A1226
:107E91006F3790FD3EB5070F126D79F9126E2D7493
:107EA10005F0A37402800D126D79F9126E2D74051F
:107EB100F0A37403F07D757F011275D190FC4AEF38
:107EC100F090FC4AE0FF60177BFF7A34794E90FD19
:107ED1003D126EF0E4F0A3EFF012A3B17F00221285
:107EE1006ED3A3F0A3F0752201E522601A90FD3E46
:107EF100126D79126E4E55226008126F6170031275
:107F01006F68126FCF80E2126F297003126F309089
:107F1100FC4EE07004A3E0640570CB90FC50E0706F
:107F210004A3E0641460327BFF7A34797B90FD3DD9
:107F3100E0126DEB12A3B1126F376F601990FD3E25
:107F4100126D79F9E490FC5AF0A3F0A37402F07D6C
:0C7F5100757F011275D17F00227F012294
:1072150090FCB3126DCC90FCB2EFF012A1D2E490C9
:10722500FF80F090FC5A126DFD127409E490FF8006
:10723500F0126E7290FC5AF0A3126FBC1275D11247
:107245006EB2C00690FCB3126D79F9126E2D126FF5
:107255007F1275D1D0E04F90FC4AF060137BFF7A26
:107265003479A890FCB2E0126DEB126F8A02734B71
:1072750090FCB3126D79F990007E12194BFFD394EF
:10728500084014126EEDE4F0A3EFF07BFF7A347939
:10729500D412A3B17F052290FCB3126D79F9900049
:1072A5007E12194B90FCB7F090007EE41219ACE405
:1072B50090FCB8F090FCB604F090FCB7E0FF90FCB1
:1072C500B6E0FED39F4003027362EEC313126DF561
:1072D50012740990FCB6E05401C433333354801260
:1072E5006DF5126FBC1275D1126EB2C006126DF932
:1072F500126F7F1275D1D0E04F90FC4AF090FF805D
:10730500E06402703190FCB8E0702B04F090FCB39F
:10731500126D792480F9E43AA801FCAD03126E726E
:107325007E007F8012190C90FCB3126D79F99000E4
:107335007E74011219AC90FC4AE0FF60177BFF7A5E
:10734500357911126EEDE4F0A3EFF012A3B190FCC4
:107355004AE0FF2290FCB6E004F00272BE90FCB356
:10736500126D79F9E412199A90FCB3126D79F990BE
:10737500000174FF1219AC90000274FF1219AC9051
:10738500000374FF1219AC90000474FF1219AC903D
:10739500000574FF1219AC90000674FF1219AC9029
:1073A5000007E41219ACE490FCB9F0126ED490FC1D
:1073B500B8E060067E017F0080047E007F80C39078
:1073C500FC4FE09FEE6480F8126F5A98501A90FCBB
:1073D500B3126D79126E4EFF90FCB9E02FF0126F6B
:1073E5002970CB126F3080C690FCB9E060137BFF2B
:1073F5007A35793D90FCB2E0126DEB12A3B17F06B0
:0F740500227F002204F0A3F07D60FF1275D122D8
:109C030090FE30126DCCED12199A90FE30126D79E0
:109C1300126EE690FCC8126DFC7402F07D007C04A9
:109C23001284A090FC4AEFF090FE30601C126D7914
:109C3300126DE77BFF7A35796412A3B190FE30127F
:109C43006D79F9900001E4802B126D79126DE79024
:109C5300FF80126E4390FF81E090FB3D126E477BC5
:109C6300FF7A35798A12A3B190FE30126D79F9909B
:089C7300000174011219AC227A
:10804D0090FDB2126DCCA3EDF090FDB2126D794A98
:10805D004B700302813490FDB2126D79126E0620C1
:10806D00E003028134126ED390FC4E126D9F741298
:10807D00126D9A74DE126D9A740FF0126E6E126E8E
:10808D00FC7D027C011284A0126ED390FDB5E0FF41
:10809D0090FC4EE475F001121A81FC748025F0F508
:1080AD008274FF3CF583EF126D9A74FF126D9AE4A2
:1080BD00F090FC4E126D9F7463126D9A7468126D80
:1080CD00817445126D9A7458126D9A7450126D9A8E
:1080DD007445126D9A7450126D9A742D126D9A74B6
:1080ED0053126D9A7470126D9A746C126D81747452
:1080FD00126D9A7474126D9A7465126D9A7472126F
:10810D006D9AE4F090FC4E126D9FE4F090FC4E12CF
:10811D006D9FE4F090FDB2126D79126E6D126EFCD2
:08812D007D097C011284A022EF
:10A0D50090FDB6126DCCA3EDF090FDB6126D794AE8
:10A0E5004B604190FDB6126D79126E0630E0351267
:10A0F5001932FF7D04129FBF90FDB9E0F52290FD56
:10A10500B6126D79F9121932126DD904F07D007C01
:10A11500051284A090FDB6126D79F9121932FF7DF2
:05A1250003129FBF22A0
:10A8DB0090FD43126DCC90FD43126D794A4B602471
:10A8EB0090FD43126D79126E0630E018121932FF8B
:10A8FB0090FD46126D79F9126E137402F07D077C90
:05A90B00011284A022EE
:107D080090FC97126DCC90FC97126D794A4B7003DA
:107D1800027E2A90FC97126D79126E0620E003020B
:107D28007E2A126D76F912193224FE60741460717D
:107D380014600D147003027E0B24046003027E2A73
:107D480090FC9D126D79F9121932601DEA494B6059
:107D58001890FC97126D79F9121932FF90FC9D1258
:107D68006D79F9126E13127E2B126D67F9126E136C
:107D780004F07D09FC1284A0126D672403126E0FB3
:107D8800127E36126D672406126E0F04F07D0BFC0E
:107D98001284A0126D67126E0D04F07D28FC027E1D
:107DA8002790FC9D126D79F9121932601DEA494B32
:107DB800601890FC97126D79F9121932FF90FC9DAA
:107DC800126D79F9126E13127E2B126D67F9126E0D
:107DD8001304F07D09FC1284A0126D672403126E4F
:107DE8000F127E36126D672406126E0F04F07D0B9B
:107DF800FC1284A0126D67126E0D7408F07D297C48
:107E080001801C126D67F9126E1304F07D0AFC12D2
:107E180084A0126D67126E0D7402F07D317C011220
:107E280084A022740EF07D127C011284A0227403B7
:097E3800F07D0F7C011284A022F0
:10A9100090FD49126DCC90FD49126D794A4B60242F
:10A9200090FD49126D79126E0630E018121932FF4F
:10A9300090FD4C126D79F9126E137403F07D0C7C4E
:05A94000011284A022B9
:10A5E70090FCBA126DCC90FCBA126D794A4B70038D
:10A5F7007F012290FCBA126D79126E0620E0037F6C
:10A60700012212193204FF90FCBD126D79F9A312D1
:0FA617006EFF7D007C071284A090FC4AEFF022BA
:1087D20090FCA0126DCC90FCA0126D794A4B7002F5
:1087E200FF2290FCA0126D79126E0620E0037F003A
:1087F20022786676000876017866E6FE08E6FFC310
:10880200940FEE9400400302888FEF64054E606F70
:1088120090FCA0126D79126EE6C007126E793402D6
:10882200FC126DDA04F0D0071284A0E522F4604F46
:10883200E522604B90FCA0126D79126EE6C0071221
:108842006E793402FC90FCA3126D79F9126E1374E6
:108852000FF0D0071284A090FCA0126D79126EE680
:10886200C007126E793403FC90FCA6126D79F912DE
:108872006E13740EF0D0071284A07867E6FF227898
:108882006706E61860030287FA060287FA7BFF7A18
:098892003579AE12A3B17F0F226B
:109F5D0090FD4F126DCC90FD4F126D794A4B7002F2
:109F6D00FF2290FD4F126D79126E0620E0037F00E7
:109F7D0022126DD504F07D507C021284A0E522F4EE
:109F8D006024E522602090FD4F126D79126EE690EF
:109F9D00FD52126D79F9126E137409F07D507C0229
:109FAD001284A07F05227BFF7A3579C912A3B17F78
:029FBD00002280
:10A86F0090FD55126DCC90FD55126D794A4B6025B8
:10A87F0090FD55126D79126E0630E01912193204DF
:10A88F00FF90FD58126D79F9126E13740FF07D0061
:06A89F007C021284A022DD
:109B8A0090FDBA126DCCA3EDF090FDBA126D794A30
:109B9A004B605A90FDBA126D79126E0630E04EE4AF
:109BAA0090FF80F0126E6E126E1304F0FDFC1284A8
:109BBA00A090FF8074FF126F2290FDBA126D791285
:109BCA006E6D126E13129BF87F0112B13090FF80F6
:109BDA007405F090FDBDE090FF81F0E4A3F090FDE4
:109BEA00BA126D79126E6D126E13129BF8227403FB
:099BFA00F07D207C011284A02200
:10A9450090FD5B126DCC90FD5B126D794A4B6024D6
:10A9550090FD5B126D79126E0630E018121932FF08
:10A9650090FD5E126D79F9126E137408F07D207CEE
:05A97500011284A02284
:109D5C0090FCA9126DCCA3EDF090FCA9126D794A80
:109D6C004B605690FCA9126D79126E0630E04A12C7
:109D7C001932FF7B017AFC79AC126E1304F0FDFCF6
:109D8C001284A090FCA9126D79F9121932FF90FC83
:109D9C00AF126D79F990FCAEE0FD126E13EDF07D13
:109DAC00007C051284A090FCA9126D79F91219326D
:0A9DBC00FF90FCADE0FD129FBF22F6
:10987B0090FE33126DCC90FE33126D794A4B700211
:10988B00C32290FE33126D79126E0620E002C322C2
:10989B00D390FC49E0942090FC48E0648094804095
:1098AB001C90FE33126D79126DE77BFF7A3579EAE6
:1098BB0012A3B1E490FC48F0A3F07868F67868E660
:1098CB00603290FE33126D79F9126DD504F07D057F
:1098DB00FC1284A030110F7868E6600116E490FC4E
:1098EB0048F0A3F0D32290FC49E004F0700690FC02
:0698FB0048E004F0C32266
:10A1D20090FE5EEFF0126ED3126F42504274047E14
:10A1E20000A807088005C333CE33CED8F9FF90FE0E
:10A1F2005EE0FDEF5D90FC4F600E126F93126D7981
:10A20200126E9E12777C800C126F93126D79126E11
:10A212009E1278E3126F297003126F3002A1DA02E4
:02A22200ACD4BA
:10A12A0090FDC1EDF090FDBE126DCC126DB37D07AE
:10A13A0012870890FDBE126D79126E0630E71490F0
:10A14A00FDC1E05403FFE52254036F6026E5225463
:10A15A00FC801290FDC1E05401FFE52254016F60BA
:10A16A0012E52254FE4FF522121932126DB77D07FD
:04A17A00128708221E
:10A4DB0090FD87EBF090FD85EFF0A3EDF0EF126DA3
:10A4EB00B612870890FD88E07002A3E0600D126F32
:10A4FB00C48002C333D8FC4222800C126FC480028A
:10A50B00C333D8FCF4522290FD85E0FFA3E0FD128B
:05A51B006DB802870885
:109FBF0090FDC2EFF0ED126F2190FDC2E0126DD84F
:109FCF0004F07D06FC1284A0EF7004E52260187F78
:109FDF000112B13090FDC5E004F0700690FDC4E0B1
:109FEF0004F0126FA140D2126FA140107BFF7A369E
:109FFF00791290FDC2E0126DEB12A3B190FDC2E099
:10A00F00FF7B017AFD79C3126E1304F07D06FC020B
:02A01F0084A01B
:1087080090FD04EF126DC7126F1A90FD04E030E07F
:108718002614FD7B017AFD7905126E2D1287C81289
:108728006EB2C00690FD04E0FD90FD06126D791250
:108738006E8FE4A3F0802990FD04E0FD7B017AFDB3
:108748007905126E2D1287C8126EB2C00690FD040C
:10875800E0FD90FD06126D79126E8FA37402F0E4AD
:10876800FF1275D1D0E04F90FC4AF090FC4AE060CF
:108778002390FC4EA3E0FF12B124126F5394804063
:1087880003126FAF126F617003126F68126F6F5030
:108798000302871290FC4AE0FF601F7BFF7A36795C
:1087A8003B126DEC90FD04126E4390FD05E0FF90C6
:1087B800FB3DE4F0A3EFF012A3B190FC4AE0FF22E6
:0A87C80004F0A3F0E4FF1275D122C3
:1084A00090FCC2EFF0A3EC126DC7126F1A90FCC2E1
:1084B000E030E02614FD7B017AFC79C3126E2D12A8
:1084C0008565126EB2C00690FCC2E0FD90FCC5123C
:1084D0006D79126E8FE4A3F0802990FCC2E0FD7BE1
:1084E000017AFC79C3126E2D128565126EB2C00638
:1084F00090FCC2E0FD90FCC5126D79126E8FA374E2
:1085000002F0E4FF1275D1D0E04F90FC4AF090FCED
:108510004AE0602390FC4EA3E0FF12B124126F5397
:1085200094804003126FAF126F617003126F681274
:108530006F6F50030284AD90FC4AE0FF60217BFF27
:108540007A36793B126DEC90FCC2126E4390FCC3FC
:10855000E0FFA3E090FB3DCFF0A3EFF012A3B190BA
:10856000FC4AE0FF227402F0A314F0E4FF1275D17C
:0185700022E8
:109E940090FE51EEF0A3EFF0ED30E013786506E6A6
:109EA4001870010690FC4B126D79F97864803A9031
:109EB400FE51E07002A3E0703C786CA6B5ED540E40
:109EC4007864760008F618E6FE08E67807C333CE11
:109ED40033CED8F9FF786CE6FDEE7864F6EF4D08E2
:109EE400F690FC4B126D79F918E6FE08E6126E56F0
:069EF400F5B475B2012275
:04004E0078680622A6
:0C8C860041FB920041FB990F41FB9A005A
:106FE00090FD73E0FBA3E0FAA3E02404F9E43AFA8D
:106FF00012193254FD12199A90FD73E0FBA3E0FAC6
:10700000A3E0F92290FB9EEFF090FB97E0FF7E005B
:10701000789F7CFB7D017B017AFF798212190C90AD
:10702000FD76E0FBA3E0FAA3E02403F9E43AFA02D8
:10703000193290FD6DE0FBA3E0FAA3E02290001569
:1070400012194BFD2290FB96F0740FA3F0E490FB15
:107050009EF090FB97E0FF7E00789F7CFB7D017B9C
:10706000017AFF79822290001C021E19740B90FC99
:10707000ADF0E4A3F0A304F0A374FBF0A3749EF0BE
:1070800022900016021E19900009121E19EA494B9F
:1070900022EBF0A3EAF0A3E9F02290FB96F0A374B0
:1070A00002F090FB99E090FB9EF090FF82E090FB55
:1070B0009FF02290FC9A7401F0A374FBF0A374A0DB
:1070C000F02290001FE4F5F0021B68900009121EE8
:1070D00019021932E490FB98F090FB9622121E19C7
:1070E00090000402194B900019021E1990001FE431
:1070F00075F001121ACFFEC3E5F02290FD4C740129
:10710000F0A374FBF0A37493F02290FB96F074014B
:10711000A3F090FB99E090FB9E2290FCBD7401F0DF
:10712000A374FFF0A37480F0221219AC7B007A00E4
:10713000790022A37401F0A374FBF0A374AF229032
:10714000000102194B90000202194B90FF82E0FFF0
:1071500090FB9FF07E0078A07CFB7D017B017AFF95
:10716000798322F0A37401F0E490FB9EF090FE3945
:107170002290FC0CF090FC097401F0A374FAF0A3C7
:107180007405F090FB9B2290FB96E090FCADF09094
:10719000FB97E090FCAEF0A374012290000302196B
:1071A0004B12199A90FD6D2290FB96F07401A3F09A
:1071B00090FF92E02254FD12199A90FE392290001D
:1071C00001E40219AC90001F121A97C32212190C85
:1071D00090FE392290000502194B90001FE475F0D3
:1071E00032121B68740722121E19E9240122121E92
:1071F00019E9240222900002E40219ACF090FF8207
:10720000E0240390FB97F02290001502194B7B01BC
:057210007AFA79052265
:10A9AC0090FD6112709190FD61E0F9A3E0FAA3E0D3
:10A9BC0090FB9BC912709290FD64E0F9A3E0FAA39E
:10A9CC00E090FD28C912709290FD61126FFB028617
:01A9DC003E3C
:107F5D0090FE3612709190FE36126FFBE412199A54
:107F6D0090FE36126FFB1271BE1271F5900003E494
:107F7D001219AC90000474401219AC900005E41273
:107F8D007129C003C002C00190FE36126FFB900034
:107F9D0006121E4912712CC003C002C00190FE369C
:107FAD00126FFB900009121E4912712CC003C00202
:107FBD00C00190FE36126FFB90000C121E4912711B
:107FCD002CC003C002C00190FE36126FFB90000F53
:107FDD00121E4912712CC003C002C00190FE361250
:107FED006FFB900012121E4990FE36126FFB90002F
:107FFD0015ED127129C003C002C00190FE36126F3B
:10800D00FB900016121E4912712CC003C002C00154
:10801D0090FE36126FFB900019121E4912712CC082
:10802D0003C002C00190FE36126FFB90001C121EA1
:10803D004990FE36126FFB90001FE4F5F0021B68AD
:06B1AB0090FB92EFF02280
:1082F30090FC6212709190FC68126FFBC003C00285
:10830300C00190FC65126FFB900009121E4990FC9E
:108313006B126FFBC003C002C00190FC65126FFBC0
:1083230090000C121E4990FC68126FFBEA494B60E7
:108333001690FC65126FFBC003C002C001A3126F4D
:10834300FB900006121E4990FC6B126FFBEA494B2F
:10835300601890FC65126FFBC003C002C00190FC63
:108363006B126FFB900006121E4990FC62126FFBAA
:10837300C003C002C001A3126FFB900019121E4973
:1083830090FC68126FFBEA494B601890FC62126F15
:10839300FBC003C002C00190FC68126FFB90001683
:1083A300121E4990FC6B126FFBEA494B601890FC5C
:1083B30062126FFBC003C002C00190FC6B126FFB23
:0783C300900016121E492272
:108A2A0090FC6E12709190FC74126FFBC003C0022E
:108A3A00C00190FC71126FFB90000F121E4990FC4E
:108A4A0077126FFBC003C002C00190FC71126FFB6A
:108A5A00900012121E4990FC74126FFBEA494B6097
:108A6A001690FC71126FFBC003C002C001A3126F03
:108A7A00FB900006121E4990FC77126FFBEA494BE5
:108A8A00601890FC71126FFBC003C002C00190FC19
:108A9A0077126FFB900006121E4990FC74126FFB4E
:108AAA00EA494B601890FC6E126FFBC003C002C00B
:108ABA000190FC74126FFB900016121E4990FC770D
:108ACA00126FFBEA494B601890FC6E126FFBC003F1
:108ADA00C002C00190FC77126FFB900016121E496B
:018AEA002269
:10B05A00C003C002C00190FD6A126FFB90001C126F
:03B06A001E49225A
:1037310090FE3912709190FE39126FFB128F175063
:103741002590FB9B126FFB123CC8126FFB1270E6B7
:10375100123CDE127035240412702B1271B5126FF7
:10376100FB740112199A90FE39126FFB12713F30EE
:10377100E61E1271BE7D4012889B90FE3912703593
:10378100240412702B1271B5126FFB740112199A75
:1037910090FE39126FFB12193214604D14607B14C4
:1037A100700302385224FE70030238882405600336
:1037B10002394990FB9B126FFB123CC8126FFB123E
:1037C10070E6123CDE126FFB127066E4FD12804D52
:1037D10090FE39126FFB1270667D0112A0D590FE2A
:1037E10039126FFB740102394690FE39126FFB12D8
:1037F1009901400302394990FE39126FFB1270C2E0
:1038010012B04790FE39126FFB1270E612AA39907E
:10381100FE39126FFB740202394690FE39126FFBBA
:103821001292D1502A90FE39126FFB1270EC94194A
:10383100EE940050030239491270C21270E6129AD6
:103841008D12B08090FE39126FFB740302394680ED
:103851002A90FE39126FFB1270E612A97AEF601BF3
:1038610090FE39126FFB1270EC9432EE940050030B
:103871000239491270C2740502394690FE39126F3D
:10388100FB1270C202394990FE39126FFB1270E6C9
:1038910012B0FEEF601490FE39126FFB1270E61247
:1038A100B18AEF90FE396020801290FE39126FFBD1
:1038B1001270E612B18AEF90FE39600C1270352455
:1038C1000412702B4402800A127035240412702BEA
:1038D10054FD12199A90FE39126FFB1271C5942C86
:1038E100E5F09401500A90001FE475F001121B1BD2
:1038F1001270E612A97AEF704F90FE39126FFB1227
:1039010071C5942CE5F09401402E1270E030E11362
:1039110012AA0D90FE39127035240412702B54FD39
:1039210012199A90FE39126FFB7D8012889B90FECE
:1039310039126FFB7402800D90FE39127035240428
:1039410012702B54FD12199A90FE39126FFB1270EE
:103951006612987B4003023B8E90FE39126FFB1278
:10396100706612711AA3E4F0A37413F012A5E79024
:10397100FF80E0B410004003023B8E903983F828A9
:1039810028730239B30239D40239DB0239E2023930
:10399100ED0239FD023A11023A36023A4C023A611D
:1039A100023A71023A86023A9F023AB5023AC502D8
:1039B1003AE41270D4041271FC90FF92E0B40F0843
:1039C10090FB9E740FF08005E490FB9EF012714B0A
:1039D100023A411270D4741980171270D4741A808B
:1039E1001090FE39126FFB7D04023B8B1270D47470
:1039F1001C127163126FFB7D40023B8B1270D474F9
:103A010006F0E4A3F090FE39126FFB7D40023B8B80
:103A110078937CFB12705D7E007F031271CD126F73
:103A2100FB1270661270FB12A91090FE39126FFB27
:103A31007D10023B8B1270D47410F0A31412704CE1
:103A41001271CD126FFB7D40023B8BE490FB98F02D
:103A510074121270451271CD126FFB7D40023B8BC7
:103A61001270D47413127163126FFB7D40023B8B91
:103A7100E490FB98F0741D1270451271CD126FFB2A
:103A81007D40023B8B1270D4741EF0A37402F0E4EB
:103A91001270A690FE39126FFB7D40023B8B1270B3
:103AA100D47415F0740612704B1271CD126FFB7D38
:103AB10040023B8B1270D47416127163126FFB7D3E
:103AC10040023B8B90FB987401F090FB96741FF0C1
:103AD100A37402F0E41270A690FE39126FFB7D40D0
:103AE100023B8B90FF811270A590FB9EE0640570F4
:103AF10047A3E0702390FE39126FFB12706690FDB0
:103B0100521270B6129F5DEF6003023B8E90FE3938
:103B1100126FFB7D80023B8B90FE39126FFB12709E
:103B21006690FD521270B6129F5DEF606090FE3993
:103B3100126FFB7D80023B8B90FB9FE0702190FE1A
:103B410039126FFB12706690FCA31270B6127133BA
:103B5100123CD2703890FE39126FFB7D80802B9021
:103B6100FE39126FFB12706690FCA31270B61271CF
:103B710033123CD2601790FB9EE0FF90FB99E0B5B9
:103B8100070B90FE39126FFB7D801297F390FE397F
:103B9100126FFB127145FD600C1297F390FE391202
:103BA1006FFB1271F590FE39126FFB12719B30E3BE
:103BB10028E912702954F71271B7126FFB1270665F
:103BC100C003740612706ED003E4FD129D5C90FE7A
:103BD10039126FFB7D080297F390FE39126FFB12C9
:103BE100719B30E42EE912702954EF1271B7126FF4
:103BF100FB1270661270FB12A91090FE39126FFB56
:103C0100127066C00390FCAD740CF0E4A3F0A30441
:103C1100023CBD90FE39126FFB12719B30E63CE90C
:103C210012702954BF12199A90FB96E0B4071A90AA
:103C3100FE39126FFB12706690FD5E7401F0A37481
:103C4100FBF0A3749FF012A94590FE39126FFB128D
:103C51007066127187127077023CC290FE39126F42
:103C6100FB12719B30E517E912702954DF1271B70D
:103C7100126FFB12706690FB99E0FD029B8A90FE29
:103C810039126FFB12719B30E73CE9127029547FA6
:103C910012199A1270D47418F0A37402F090FB9E5A
:103CA10014F0E4A3F090FE39126FFB127066C003AA
:103CB10090FCAD7418F0A37402F0A314127077D0C5
:103CC10003E4FD129D5C2212923512B04790FE3939
:103CD10022F01287D290FB99EFF0640F2212AA39D9
:043CE10090FE3922F6
:1056060090FD6D127091900006121E1990FD701299
:10561600709190FD6D126FFB128F17400E90FD6D0D
:10562600126FFB12713F700302570290FD6D126FED
:10563600FB127081C003C002C00190FD6D126FFBAA
:1056460012703DD001D002D00312AE6E1270322419
:105656000412702B54FD1271A1126FFB127081C0DF
:1056660003C002C00190FD6D126FFB12703DD001A8
:10567600D002D00312ADA990FD6D126FFB1270819E
:10568600C003C002C00190FD6D126FFB12703DD0C9
:1056960001D002D003125A00126FFB1270E612AA52
:1056A6003990FD6D126FFB1270C212713F30E70A1E
:1056B60090FD6D126FFB7D80802190FD6D126FFB5A
:1056C60012713F30E62290FD70127035240112707F
:1056D6002B44401271A1126FFB7D4012889B90FDF6
:1056E6006D126FFB7402800890FD6D126FFB7401E2
:1056F60012199A90FD6D126FFB1271BE90FD6D121C
:105706006FFB1219321470030258BB14700302584F
:10571600D41470030258ED14700302596014700318
:1057260002596A2405600302599D127081C003C0A4
:1057360002C00190FD6D126FFB12703DD001D002C8
:10574600D003125A00126FFB1270E612AA3990FDAE
:1057560070126FFB12193270411271D490FD6D30C8
:10576600E40C127035240512702B4410800A127056
:1057760035240512702B54EF12199A90FD70126F92
:10578600FB1271D490FD6D30E50302586912703535
:10579600240512702B54DF0258731270322405123E
:1057A600702B54EF12199A54DF1271A1126FFB126B
:1057B6007081C003C002C00190FD6D126FFB1270B4
:1057C6003DD001D002D00312AD6790FD6D126FFB84
:1057D6001270E6129A8D90FD6D126FFB127081C0E9
:1057E60003C002C00190FD6D126FFB12703DD00127
:1057F600D002D00312A665EF700D12703224051286
:10580600702B441002587390FD6D126FFB1270815D
:10581600C003C002C00190FD6D126FFB12703D9077
:10582600FCEC12711DD001D002D003128E72EF7003
:105836000C127032240512702B4410803012703214
:10584600240512702B54EF12199A90FD6D126FFBFE
:10585600127208FF7B017AFF7980128BABEF701012
:1058660090FD6D127035240512702B442002199A92
:10587600127032240512702B54DF12199A90FD6DA6
:10588600126FFB127081C003C002C00190FD6D1241
:105896006FFB12703DD001D002D00312AE4E90FDC8
:1058A6006D126FFB1270E612AA3990FD6D126FFB36
:1058B600740102599890FD6D126FFB129901400315
:1058C6000259A690FD6D126FFB740202599890FD65
:1058D6006D126FFB1292D140030259A690FD6D1214
:1058E6006FFB740302599890FD70126FFB12193208
:1058F600D3940350030259A690FD6D126FFB1270EC
:1059060081C003C002C00190FD6D126FFB12703D95
:10591600D001D002D00312AD6790FD6D126FFB125D
:1059260070E6129A8D90FD6D126FFB127081C003A6
:10593600C002C00190FD6D126FFB12703DD001D008
:1059460002D00312ADEB127032240412702B440104
:105956001271A1126FFB7404803890FD6D126FFBFB
:105966007405802E90FD70126FFB1270E090FD6D35
:1059760030E115127035240412702B44021271A105
:10598600126FFB1271DA800A127035240412702B22
:1059960054FD12199A800990FD6D126FFB1247880B
:1059A60090FD6D126FFB129A0C127032500924048E
:1059B60012702B44108007240412702B54EF121916
:1059C6009A90FD6D126FFB127145FD600C1297F3F4
:1059D60090FD6D126FFB1271F590FD6D126FFB124B
:1059E600719BFF601490FD701270224F1271A1120C
:1059F6006FFB900003E41219AC2212AE4E90FD6DBF
:015A0600227D
:1023740090FD73127091900006121E1990FD761252
:102384007091126FF8121932D39401500302246031
:10239400127081C003C002C001126FF812703DD0E8
:1023A40001D002D003129CF2EF6011126FF8127088
:1023B400E020E50812713F7003022460126FF812E6
:1023C4007081C003C002C001126FF812703DD001C9
:1023D400D002D00312AE6E126FE0127081C003C03F
:1023E40002C001126FF812703DD001D002D0031266
:1023F400ADA9126FF8127081C003C002C001126F40
:10240400F812703DD001D002D00312AE4E126FF814
:102414001270C212713F30E72B126FF8127081C034
:1024240003C002C001126FF812703DD001D002D077
:1024340003129CF2EF90FD736005126FFB800E1285
:102444006FFB800D126FF812713F30E60474028046
:1024540002740112199A126FF81271BE126FF812F7
:102464001932B4070040030228B9902475F82828CB
:102474007302248A0225C20227500227680227DA3F
:102484000227EB022847127081C003C002C0011268
:102494006FF812703DD001D002D00312AE4E90FD01
:1024A40076126FFB121932704B1271D490FD733097
:1024B400E40C127035240512702B4410800A12703B
:1024C40035240512702B54EF12199A90FD76126F71
:1024D400FB1271D490FD7330E50D12703524051292
:1024E400702B4420022583127035240512702B545E
:1024F400DF02258390FD73127035240512702B546E
:10250400EF12199A54DF126FF5127081C003C002E2
:10251400C001126FF812703DD001D002D00312AD89
:1025240067126FF8127081C003C002C001126FF805
:1025340012703DD001D002D00312A665EF700F9047
:10254400FD73127035240512702B44108031126F04
:10255400F8127081C003C002C001126FF812703DFE
:1025640090FCEC12711DD001D002D003128E72EFD8
:10257400701090FD73127035240512702B441002F4
:10258400199A90FD73127035240512702B54EF12B2
:10259400199A126FF8127081C003C002C001126F41
:1025A400F812703DD001D002D00312AE4E126FF873
:1025B4001270667D0412804D126FF802294E126F5C
:1025C400F8127081C003C002C001126FF812703D8E
:1025D400D001D002D003129CF2EF700302295B12E7
:1025E4006FF81270E030E50302295B90001FE47578
:1025F400F001121ACFFCC3E5F0940AEC94005003E6
:1026040002295BEFB4020E1271C59432E5F0940016
:10261400500302295B127208FF12720E127215EF38
:10262400601B126FF81271C59419E5F09400500301
:1026340002295BE9240512702B4440800D90FD7340
:10264400127035240512702B54BF12199A126FF8A8
:102654001270C212720E1295C3EF90FD73604B128A
:102664007035240412702B440112199A12720E123E
:102674009DC674092FF974FA3EFA90FD467401124E
:102684007092126FF812706612A8DB126FF8127053
:10269400667D0212A0D5126FF8127066C003127024
:1026A4006CD003E4FD129D5C800D1270352404127D
:1026B400702B54FE12199A126FF8127066E94A4B85
:1026C4006038126FF812706612713F30E02C126F8E
:1026D400F812708112B0FEEF600D126FF81270E004
:1026E40030E6047F0180027F00EF4404127171120E
:1026F4006FFB120280EF604F803D126FF812708101
:1027040012B0FEEF600D126FF81270E030E6047F35
:102714000180027F00126FF8127208FE90FB92E0B3
:10272400B506047E0280027E00EE4F127171126FB4
:10273400FB120280EF601090FD76127035240112B6
:10274400702B444012199A126FF88013126FF8120A
:1027540070EC940AEE9400500302295B1270C27468
:102764000302295090FD76126FFB121932D39403A1
:10277400500302295B126FF8127081C003C002C0BB
:1027840001126FF812703DD001D002D00312AD6770
:10279400126FF81270E030E01A127081C003C002A8
:1027A400C001126FF812703DD001D002D00312ADF7
:1027B400EB801B126FF8127081C003C002C00112BB
:1027C4006FF812703DD001D002D00312AE8E126F9A
:1027D400F87404022950126FF812708112A757126C
:1027E4006FF87405022950126FF8127081C003C08B
:1027F40002C001126FF812703DD001D002D0031252
:102804000026EF7026126FF8127081C003C002C058
:1028140001126FF812703DD001D002D00312AE4EF7
:10282400126FF81270C2740602295090FD76126F6E
:10283400FB1270E020E10302295B126FF81271DAD7
:10284400022950126FF81270EC94FAEE94005003BF
:1028540002295B1270C2127081C003C002C001124F
:102864006FF812703DD001D002D00312AD6712ACE4
:10287400D4126FF8127081C003C002C001126FF845
:1028840012703DD001D002D003120026EF6008126E
:102894006FF8740312199A126FF8127081C003C092
:1028A40002C001126FF812703DD001D002D00312A1
:1028B400AE4E02295B126FF8127081C003C002C0D1
:1028C40001126FF812703DD001D002D0031200261D
:1028D400EF6020126FF8127081C003C002C00112B1
:1028E4006FF812703DD001D002D003129CF2EF6455
:1028F40001605E126FF8127081C003C002C0011241
:102904006FF812703DD001D002D00312AE6E126F78
:10291400E0127081C003C002C001126FF812703D52
:10292400D001D002D00312ADA9126FF8127081C089
:1029340003C002C001126FF812703DD001D002D062
:102944000312AE4E126FF81270C2740112199A80FB
:1029540006126FF8124788126FF8121932FF640CCE
:102964006019EFD394024013EF6406600E90F9FFF0
:10297400E020E70790F9FEE030E30AE9240412704E
:102984002B4410800D90FD73127035240412702BAB
:1029940054EF12199A126FF812706612987B400362
:1029A400022BF2126FF812706612711AA3E4F0A3EC
:1029B4007413F012A5E790FF80E0121EA22A010012
:1029C4002A41032A4C052A54062A76072A9E082AF5
:1029D400BD092ADB0C2AFD0D2B2C102B34112B499D
:1029E400122B57132B72142B57152B83162B90175E
:1029F4002B9D182BB0192BBF1A00002BF290FF92BD
:102A0400E0FDB405047E0180027E0090FB98EEF0A8
:102A140090FB9674011271FCEDB4050890FB9E7452
:102A240005F0801390FF92E0B40F0890FB9E740FA2
:102A3400F08004127112F012714B022A9690FB96E8
:102A4400741BF0E4A3022AD212701F4408022BEF75
:102A540078937CFB12705D7E007F0312190C126F59
:102A6400F81270661270FB12A91012701F44100243
:102A74002BEF90FB967410F0A314F090FF92E0B447
:102A840005047F05800590FB99E0FF90FB9EEF1203
:102A9400705112701C4440022BEF90FB967412F09C
:102AA400740F1271AEB405047F05800590FB99E0A4
:102AB400FF1270044440022BEF74131271A8B40582
:102AC400047F05800590FB99E0FF90FB9EEFF012D8
:102AD400701F4440022BEF90FB967415F0A374060C
:102AE400F090FF92E0B405047F05800590FB99E027
:102AF400FF1270044440022BEF74161271A8FFB445
:102B040005047E05800590FB99E0FE90FB9EEEF0A7
:102B140012701F444012199AEF64056003022BF2ED
:102B240012701F4480022BEF12701F4420022BEFFF
:102B3400740712710AF01270597E007F0812701C1B
:102B44004440022BEF740812710AF012701F4440C3
:102B5400022BEF90FB967409F07411127110F012AD
:102B640070597E007F1012701C4440022BEF78AF26
:102B74007CFB12705D7E007F0E12190C022BF27426
:102B84001412709A12701F4440022BEF740D1270CD
:102B94009A12701F4440022BEF90FB96740EF0A320
:102BA40074091271111270084440803F90FB9674AE
:102BB4000F12709D12701F4440803090FB96741762
:102BC400F0A37403F090FB9E74051270A990FF8427
:102BD400E0600790FB99E0FF80027F0090FBA0EF8C
:102BE400F012701F444012199A448012199A126FFD
:102BF400F812714530E127E9240212702B54FD12BA
:102C0400199AE490FB9EF0126FF812706690FCAD76
:102C1400741AF0A37401F0A3127077022D56126F88
:102C2400F812714530E21DE9240212702B54FB1294
:102C34006FF5127066C00390FCAD741B127071D0F6
:102C440003022D56126FF812714530E31DE9240278
:102C540012702B54F7126FF5127066C00390FCAD1E
:102C64007406127071D003022D56126FF81271455A
:102C740030E429E9240212702B54EF126FF512701C
:102C8400661270FB12A910126FF8127066C00390DE
:102C9400FCAD740C127071D003022D56126FF81231
:102CA400714530E61CE9240212702B54BF126FF5F3
:102CB40012706690FB98E0FD127187127077022DF6
:102CC40089126FF812714520E703022D9CE9240252
:102CD40012702B547F12199A90FB9EE06405704287
:102CE400A3E064047015126FF81270661270B3A337
:102CF400E4F0A3F0A3F0127D08800A90FB9FE0703B
:102D04000FA374FFF0126FF81270667D0202A0D553
:102D1400126FF81270661270B3A3E4F0A3F0A3026A
:102D24002D9890FB9FE06404702C126FF81270666B
:102D34001270B3127133F0127D08126FF8127066BC
:102D44007D0212A0D5126FF8127066C00312706C67
:102D5400D003E4FD802F90FB9FE0702CA37404F05B
:102D6400126FF81270667D0412804D126FF81270A3
:102D7400667D0212A0D5126FF8127066C00312703D
:102D84006CD003E4FD029D5C126FF8127066127041
:092D9400B3127133F0127D082224
:0BB15400E9240412702B442002199A19
:0BB15F00E9240412702B54DF02199A3F
:108F170090FE3C12709190FE3C126FFB121932D3F7
:108F270094014003D38001C340012212708760136C
:108F370090FE3C126FFB1270CBB40103D38001C3C8
:108F470040012290FE3C126FFB90000C12708A6069
:108F57001690FE3C126FFB90000C1270CEB401030A
:108F6700D38001C340012290FE3C126FFB90000F9B
:108F770012708A601690FE3C126FFB90000F127001
:108F8700CEB40103D38001C340012290FE3C126F8F
:108F9700FB90001212708A601690FE3C126FFB90D5
:108FA70000121270CEB40103D38001C3400122D353
:018FB7002297
:1099010090FE3F12709190FE3F126FFB12708760C4
:109911001090FE3F126FFB1270CBD394014002D323
:109921002290FE3F126FFB90000C12708A60139020
:10993100FE3F126FFB90000C1270CED394014002D7
:10994100D32290FE3F126FFB90000F12708A6013BA
:1099510090FE3F126FFB90000F1270CED394014026
:1099610002D32290FE3F126FFB90001212708A60A8
:109971001390FE3F126FFB9000121270CED3940130
:069981004002D322C322C4
:1092D10090FE4212709190FE42126FFB12708760F5
:1092E1001590FE42126FFB1270CBFF64036007EF13
:1092F100D3940140012290FE42126FFB90000C12A8
:10930100708A601890FE42126FFB90000C1270CEB2
:10931100FF64036007EFD3940140012290FE4212E3
:109321006FFB90000F12708A601890FE42126FFB63
:1093310090000F1270CEFF64036007EFD3940140D9
:10934100012290FE42126FFB90001212708A601887
:1093510090FE42126FFB9000121270CEFF64036008
:0A93610007EFD39401400122D3224C
:109A0C0090FE4512709190FE45126FFB12708760AC
:109A1C001190FE45126FFB9000091270DD20E402DC
:109A2C00C32290FE45126FFB90000C12708A6011DD
:109A3C0090FE45126FFB90000C1270DD20E402C307
:109A4C002290FE45126FFB90000F12708A601190ED
:109A5C00FE45126FFB90000F1270DD20E402C32252
:109A6C0090FE45126FFB90001212708A601190FEEE
:109A7C0045126FFB9000121270DD20E402C322D35A
:019A8C0022B7
:10889B0090FE4812709190FE48126FFB1270876029
:1088AB002190FE48126FFB1270CBD39403401390B0
:1088BB00FE48126FFB9000091271E712702B4D12DC
:1088CB00199A90FE48126FFB90000C12708A60246C
:1088DB0090FE48126FFB90000C1270CED3940340A5
:1088EB001390FE48126FFB90000C1271E712702B65
:1088FB004D12199A90FE48126FFB90000F12708A5E
:10890B00602490FE48126FFB90000F1270CED39430
:10891B0003401390FE48126FFB90000F1271E71289
:10892B00702B4D12199A90FE48126FFB9000121289
:10893B00708A602490FE48126FFB9000121270CE6A
:10894B00D39403401390FE48126FFB9000121271E8
:09895B00E712702B4D12199A224B
:1097F30090FE4B12709190FE4B126FFB12708760BC
:109803001390FE4B126FFB9000091271EE12702B36
:109813004D12199A90FE4B126FFB90000C12708A36
:10982300601390FE4B126FFB90000C1271EE1270DE
:109833002B4D12199A90FE4B126FFB90000F127072
:109843008A601390FE4B126FFB90000F1271EE12A1
:10985300702B4D12199A90FE4B126FFB900012124F
:10986300708A601390FE4B126FFB9000121271EE20
:0898730012702B4D12199A220C
:108C9200182F00000000000000000000000000008B
:0A8CA20000000000000000000000C8
:10A2240085128385138222860308E6FA08E64A4BE0
:10A234002208E6FA08E6F9021EC8A3E0FEA3E0FF3E
:10A244002290FFFF121ECEEFF0C2A922AA06AB078E
:10A2540090FE5FE025E0227C001219E0EF22F8A6D0
:10A264000308A60208A60122F8E6FE08E6FFE4FCBD
:02A27400FD22C9
:10006E0090FFFF121ECEEBF090FFFE121ECEECF0B4
:10007E00A3EDF012A245E58954FCFE12A224E0FB8A
:10008E004EF589900003121EF2E044C0F58B90FEEF
:10009E0063E014605A1470030201452402600302E7
:1000AE00019712A22412A23EEE54FE7009758C1610
:1000BE00EEC313EF805F12A22412A23EEE54FC7028
:1000CE0010758C2DEF7802CEC313CE13D8F9020122
:1000DE008612A22412A23ED394EAEE9415500B750A
:1000EE008CFC7D1612A25B020186AF0302019012F8
:1000FE00A224A3E0FEEE700C758C0E12A224A3A314
:10010E00E0020186EE54FE700F758C1D12A224A320
:10011E00E0C313A3E013806012A22412A23ED39474
:10012E00EFEE9410500A758CFE7D1112A25B804882
:10013E0012A224E0FF804B12A224A3E0FEEE700B6D
:10014E00758C1012A224A3A3E0802DEE54FE700F26
:10015E00758C2112A224A3E0C313A3E013801912FD
:10016E00A22412A23ED394EFEE94105010758CFE82
:10017E007C007D0F1219E0EF14F58D800C12A22475
:10018E00E0FF12AECD7F00803CAF8C12A224E0FDCA
:10019E0025E02427F8760008A607AF8DED25E0248C
:1001AE0047F8760008A6077401A805088002C33335
:1001BE00D8FCF5887410A805088002C333D8FC4219
:0B01CE0089D2A97F01900004021ECE20
:10AECD0012A24512A224E0FF7410A807088002C345
:0EAEDD0033D8FCF45289D2A9900001021ECE97
:0BB16A00EF75F003A4242F12A2622254
:0BB17500EF75F003A4243B12A262223D
:1089640090FE5FEFF0FBC2A9E58954FC4BF589AF9B
:108974008C7862760008A607AF8DE4FCFDFE785E75
:10898400121DD0EB25E0244712A26C785E121D93D1
:10899400C3EF9BFFEE9AFEED99FDEC98FCC004A991
:1089A4000512A250242712A26CD000121B95C004F9
:1089B400C00512A2502428F9C3E7786396FF19E78B
:1089C4001896FEE4FCFDD001D000EB2FFFEA3EFE3A
:1089D400ED39FDEC38FC785E121DD090FE63E01496
:1089E400601C14602424027033E47F19FEFDFC78BB
:1089F4005E121D93121B95E47B207A018014785E2D
:108A0400121D87E47B0FFA8009785E121D87E47BD0
:108A140011FAF9F8121C20785E121DD0D2A97860E0
:068A2400E6FE08E6FF2259
:03000B0002821A54
:10821A00C0E0C0F0C083C082C0D075D000C000C02A
:10822A0001C002C003C004C005C006C007308812DE
:10823A00782F12A22B6005782F12A23575880102B9
:10824A0082D8308912783212A22B6005783212A2B3
:10825A00357588020282D8308A12783512A22B60CC
:10826A0005783512A2357588040282D8308B1178C8
:10827A003812A22B6005783812A235758808804E0C
:10828A00308C11783B12A22B6005783B12A235750F
:10829A008810803A308D11783E12A22B6005783E04
:1082AA0012A2357588208026308E11784112A22BB1
:1082BA006005784112A2357588408012308F0F7898
:1082CA004412A22B6005784412A235758880D00723
:1082DA00D006D005D004D003D002D001D000D0D02F
:0982EA00D082D083D0F0D0E03244
:08B19300E5FF54077869F6227C
:0500060012B19300227D
:10AEEB0012B193E6FF700476098008EFB4010C7879
:0CAEFB006976027869E660031680F82290
:10AD440012B193E6FF7004760C800FEFB40106781D
:10AD54006976048005EFB40209227869E660031677
:03AD640080F82252
:10ACD40012B193E6FF700476178012EFB401067880
:10ACE4006976098008EFB4020C786976027869E61F
:06ACF40060031680F82247
:10A3640090FE63E014601314602624027036E5FF47
:10A37400540770387869760D802AE5FF5407146015
:10A384000904702878697615801A78697603801430
:10A39400E5FF54071460090470127869761A800482
:0DA3A400786976057869E660031680F82276
:109B0C0090FE63E014602714604424027067E5FF44
:109B1C00540714600D146010240270617869764546
:109B2C0080537869761B804D786976058047E5FF10
:109B3C00540714600D146010240270417869765F2C
:109B4C00803378697628802D7869760C8027E5FF3C
:109B5C0054071460101460131460162403701E78DC
:109B6C0069766D80107869762F800A7869760F8017
:0E9B7C0004E47869F67869E660031680F82242
:10940400303204D2AED2BE90FE63E01460301460F9
:109414005624027079E5FF54071460101460131485
:109424006016240370707869767E80627869763776
:10943400805C786976138056786976018050E5FF00
:1094440054071460101460131460162403704778D2
:109454006976A980397869764C80337869761E807C
:109464002D786976078027E5FF540714601014608F
:10947400131460162403701E786976C0801078690E
:109484007658800A7869762480047869760A78693F
:07949400E660031680F822D8
:107A4A00303204D2AED2BE90FE63E0146078147075
:107A5A0003027B3A24026003027B99E5FF5407B4D0
:107A6A0007004003027BA9907A78F8282873027AE3
:107A7A008D027A94027A9E027AA8027AB2027ABCBB
:107A8A00027AC6786A7603027B2C786A76010876CF
:107A9A0084027B99786A76000876BC027B99786AB8
:107AAA007600087658027B99786A7600087626026C
:107ABA007B99786A760008760D027B99786A760057
:107ACA00087601027B99E5FF5407B40700400302D8
:107ADA007BA9907AE3F8282873027AF8027B0202DB
:107AEA007B0C027B16027B1F027B28027B31786AA1
:107AFA007604087607027B99786A76010876FD0291
:107B0A007B99786A76000876F9027B99786A76001A
:107B1A00087676807A786A76000876358071786A8F
:107B2A0076000876158068786A7600087604805FA1
:107B3A00E5FF5407B407005066907B4AF82828737B
:107B4A00027B5F027B68027B71027B77027B800289
:107B5A007B89027B92786A76040876898031786A12
:107B6A00760208763E8028786A76018016786A76E8
:107B7A00000876878019786A760008763D80107842
:107B8A006A76000876198007786A76000876067899
:107B9A006BE61846600908E6161870F31680F0229C
:10B0B4007869760A7869E6166005127A4A80F5227C
:10B0C400786976647869E6166005127A4A80F52212
:0CB11800AE071FEE600512940480F522C3
:0CB12400AE071FEE6005127A4A80F5228B
:0CB13000AE071FEE600512B0B480F522DF
:0CB13C00AE071FEE600512B0C480F522C3
:108CAC000F4F00000000000000000000000000005A
:018CBC0000B7
:10AB920090FFFF121ECEEFF085128385138222866C
:10ABA2000308E6FA08E64A4B2208E6FA08E6F90242
:0AABB2001EC8E0FF7401A807082286
:10A6260090FFFF121ECEEDF012AB9212ABB4800279
:10A63600C333D8FC12AB9AF0E0FF42F312AB9AA3F5
:10A64600E06005EF42F4800712AB9AE0F452F41290
:0FA65600AB9AE0F5F6D2A842F5900002021ECEB4
:10AF230012AB9212ABB48002C333D8FC12AB9AF0CB
:0AAF3300E055F2FF900001021ECE6F
:10AFE10012AB9212ABB48002C333D8FCF452F59089
:05AFF1000001021ECE6C
:10B09200EF75F003A4244FF8A60308A60208A60140
:01B0A200228B
:030003000290590F
:10905900C0E0C0F0C083C082C0D075D000C000C0DD
:1090690001C002C003C004C005C006C007E5F5552C
:10907900F6F523301811784F12ABA16005784F121D
:10908900ABAB75F601804E301911785212ABA16065
:1090990005785212ABAB75F602803A301A11785541
:1090A90012ABA16005785512ABAB75F6048026307A
:1090B9001B11785812ABA16005785812ABAB75F645
:1090C900088012301C0F785B12ABA16005785B1227
:1090D900ABAB75F610D007D006D005D004D003D0BD
:1090E90002D001D000D0D0D082D083D0F0D0E032ED
:088CBD00061400000000000095
:1095320075BC01C390FC60E094A890FC5FE094616C
:1095420022781408E6FA08E6F5828A83021ECC78AD
:1095520014860308E6FA08E64A4B2290FC5AE0FE1B
:10956200A3E0FF90FC5DE0FCA3E0FDC39FEC9E2224
:10957200F5B7E490FC5FF0A3F022E5BC540690FC42
:1095820061F022ED5401C4333354C022781C080622
:10959200E6188606222453F582E434FEF5832290EF
:1095A200FC5FE004F02290FC617403F022E490FC82
:1095B2005DF0A3F02290FC57E0FBA3E0FAA3E0F9F0
:0195C2002286
:10A8A500EF6019D2BAED6006D2B6D2B78004D2B441
:10A8B500D2B543BB04E490FE54F08017D2B9ED60E5
:10A8C50006D2B2D2B38004D2B0D2B143BB02E49077
:06A8D500FE53F002AB137C
:10AB1300EF600543BB01800353BBFEEDB4020CEBB6
:10AB23005403C454F0FF129585800C12958544801C
:0BAB3300FFEB5403C454F04FF5B722B1
:10A6DF0090FDC8EBF0EF6014D2BAED6006D2B6D29F
:10A6EF00B78004D2B4D2B543BB048012D2B9ED60A7
:10A6FF0006D2B2D2B38004D2B0D2B143BB0212ADF4
:0CA70F002090FDC8E0F5B3A3E0F5B622F1
:10AD2000E5BB54FE4FF5BBEDB40208129586442EE8
:10AD3000F5B12212958544AEF5B175B4FF75B21F19
:04AD400043B10122F8
:10B0A300EF75F003A42414F8A60308A60208A6016A
:01B0B300227A
:1075D10090FC55EFF0A3EDF0A3EBF0A3EAF0A3E9E3
:1075E100F01295AFA3F0A3F0A3F090FC55E0FE12CA
:1075F1009597E060037F012274532E1295997401CF
:10760100F0E5BB54FE4EF5BB75BC0190FC5CE0207F
:10761100E12E90FC56E0F5BDE5B754F14402129518
:1076210072E5BC20E00D12776870031295A11295E6
:107631003540EE129532500512957C80031295A8C3
:1076410090FC61E0600302775990FC56E020E00372
:107651000276D71295AF12955D400302772A90FC0E
:1076610061E0600302772AEF24FFFFEE34FFFEEDB5
:10767100B50715ECB5061190FC5CE020E00AE5B712
:1076810054F1440AF5B78008E5B754F14406F5B75B
:10769100129574E5BC20E00D12776870031295A174
:1076A10012953540EE1295B790FC5DE0FEA3E0F532
:1076B100828E83E5BF1219AC129532500512957C6A
:1076C10080031295A890FC5EE004F0700690FC5DCA
:1076D100E004F00276571295AF12955D504B90FC85
:1076E10061E070451295B78D828C8312194BF5BEFE
:1076F100E5B754F14406129572E5BC20E00D12770E
:107701007270031295A112953540EE129532500513
:1077110012957C80031295A890FC5EE004F070063F
:1077210090FC5DE004F00276DA90FC5CE020E02859
:10773100E5B754F1440E129572E5BC20E00D1277C5
:107741007270031295A112953540EE1295325005D3
:1077510012957C80031295A890FC55E0129597E450
:10776100F090FC61E0FF2212000690FC60E004F062
:0B7771002212000690FC60E004F022F1
:03004B00028D1C07
:108D1C00C0E0C0F0C083C082C0D075D000C000C01D
:108D2C0001C002C003C004C005C006C00790FE60AD
:108D3C00E5BBF053BBFEE5B230E119129551600F63
:108D4C0012958E70010614FF781AE6FD1295437584
:108D5C00B202804AE5B230E211781AE620E006440D
:108D6C0001F675B20175B2048034E5B230E31078C7
:108D7C001C7600087600781AA6B575B208801FE537
:108D8C00B230E01A781AE6FD30E013129551600B00
:108D9C0012958E70010614FF12954375B20190FE68
:108DAC0060E0F5BBD007D006D005D004D003D002CC
:0F8DBC00D001D000D0D0D082D083D0F0D0E03220
:03005300028AEB33
:108AEB00C0E0C0F0C083C082C0D075D000C000C051
:108AFB0001C002C003C004C005C006C00790FE61E0
:108B0B00E5BBF0E5BB54FE4401F5BBE5B230E11F1C
:108B1B0078171295536013781E12959070010614F6
:108B2B00FF781BE6FD781712954575B2028050E56C
:108B3B00B230E211781BE620E0064401F675B20173
:108B4B0075B204803AE5B230E310781E76000876F1
:108B5B0000781BA6B575B2088025E5B230E0207809
:108B6B001BE6FD30E0197817129553600F781E1233
:108B7B00959070010614FF781712954575B2019008
:108B8B00FE61E0F5BBD007D006D005D004D003D0F2
:108B9B0002D001D000D0D0D082D083D0F0D0E03240
:10AC0F00EBF0A3EAF0A3E9F02290FD99E0FBA3E0BB
:10AC1F00FAA3E0F92275A102439A03439C03539BC5
:09AC2F00FC227B017AFF798022EE
:108FB80090FD8AEEF0A3EFF0A3EDF090FE63E014CD
:108FC800600F146014240270507F007ED07D0280F0
:108FD8000E7F807EA97D0380067FB07E1E7D047C87
:108FE80000E5FF5407F9F8121CD2E47B20FAF9F8DF
:108FF80012A520C006C00790FD8AE0FEA3E0FBAAE8
:1090080006E4F9F8D007D00612A520C3E49F90FD26
:109018008EF074049E90FD8DF04387807598509073
:10902800FD8DE0F5BAA3E0F5AA75A101E5A1B401AB
:109038000512AC2480037595037E007F127D007BAA
:10904800017AFC793612224E90FD8CE06002D2AC97
:0190580022F5
:10A2760090FD8F12AC0FA3ECF0A3EDF0E4FFFE759A
:10A28600A101E5A1B4010512AC248003759503D3A1
:10A2960090FD93E09FEE6480F890FD92E0648098D4
:10A2A600401E90FD8F12AC1B8F828E8312194BF5C8
:10A2B60099E59830E1FB5398FD0FBF00010E80CF62
:01A2C6002275
:10AF550090FE62EFF07B017AFE79627D017C001242
:08AF6500A27690FE62E0FF22DB
:10A71B0090FD9412AC0FE4A3F0A3F090FD9412AC57
:10A72B001BA3E0FEA3E0F5828E8312194BFF60138F
:10A73B0012AF5590FD98E004F070E090FD97E004A7
:0CA74B00F080D890FD97E0FEA3E0FF2214
:10A3B10090FB3612AC0F90FB617401F0A374FBF0BB
:10A3C100A37439F090FB36E0F9A3E0FAA3E090FD25
:10A3D1007FC912AC1090FB61E0F9A3E0FAA3E09011
:10A3E100FD82C912AC1012AC3112A44B12AC311265
:0DA3F100AFF6AC06AD0712AC3112A2762219
:0300230002A17EB9
:10A17E00C0E0C083C082C0D075D000C004C005C08E
:10A18E0007E59830E02F90FC46E0FF2401FDE43314
:10A19E00FCA3E06D7001EC601974362FF582E43487
:10A1AE00FCF583E599F090FC46E004F0E0B4100273
:10A1BE00E4F05398FED007D005D004D0D0D082D092
:04A1CE0083D0E03228
:10AC5F007FFF90FC47E0FE90FC46E06E6018743674
:10AC6F002EF582E434FCF583E0FF90FC47E004F01E
:07AC7F00E0B41002E4F02232
:10A07F0090FD9912AC0FA3ECF0A3EDF0E4FDFCD32F
:10A08F0090FD9DE09DEC6480F890FD9CE0648098CD
:10A09F00402F12AC5FEFF460F912AC188D828C83F5
:10A0AF00EF1219ACEFB40A12ED1D70011C12AC18AF
:10A0BF008D828C83E41219AC80070DBD00010C80DA
:06A0CF00BEAE04AF052245
:108CC5004DFC27000000FF000000000000F0E00060
:108CD50041FC230041FC240041FC340041FC3500EB
:088CE50041FC260041FC2200C5
:10998700C454F0FEEF4EFFF090FE4EE02427F58220
:10999700E434FCF58322E0FF90FE4FE022E0FE90E6
:1099A700FE5AE022E090FE56FEE033333354F822AD
:1099B70075A101E5A1640122E090FE4FFEE0C454C9
:1099C700F0FD22E0FD90FE5AE0FCED6C22E0FF2462
:1099D700FB24FB22C454F0FD90FC22E05DFDEE2247
:1099E70090FE5AE0FFEE6F2290FE4FE0540FF0A377
:1099F700E0FF22E0FEC454F05FFFEE4FF022F4FEDA
:059A0700EF5EF0EE220D
:1067D20090FE4FEDF0A3EBF090FE4EEFF014604907
:1067E2001460791470030268841470030268A3248D
:1067F200FA70030268D614700302691D240B600349
:1068020002698490FE50E0FF700790FE4FE042FC68
:1068120022EF90FE4FB40205E042C88004E0F45239
:10682200C890FE4FE0F452FC2290FE50E0FF700749
:1068320090FE4FE042FD22EF90FC23B40212129927
:106842009DFEEF4EFF90FC2312998EE05F42FD22E7
:1068520012999D90FC23129A0552FD2290FE50E05F
:10686200FF700790FE4FE042FE22EF90FE4FB4020F
:1068720005E042D88004E0F452D890FE4FE0F45292
:10688200FE2290FE50E0701212998FC083C08212D5
:10689200999DFEEF4ED082D083F012998FE0F5B031
:1068A2002290FE50E0FF700790FE4FE042F322EF8D
:1068B20090FC24B4021212999DFEEF4EFF90FC242C
:1068C20012998EE05F42F32212999D90FC24129A53
:1068D2000552F3221299EF701312998FC083C0826E
:1068E2001299BFEE4DD082D083F08028EF90FC3415
:1068F200B4020E12999D90FC341299871299FA8073
:106902001312999DC454F0F4FEEF5E90FC34129978
:106912008EE05EF012998FE0F58A2290FE4FE054ED
:106922001CF0A3E0FF701812998FC083C082E09020
:10693200FE4F1299AFFDEE4DD082D083F0803CEF36
:1069420090FC35B4022012999D33333354F8FEEF94
:106952004EFF90FC3512998EE0FE33333354F85FCC
:10696200FFEE4FF0801512999D33333354F8F4FE45
:10697200EF5E90FC3512998EE05EF012998FE0F591
:10698200C1221299B7706E90FE4E1299D45007240C
:10699200FE602C026AAD12ACFA90FE50E0FF700766
:1069A20090FE4FE0429B22EF90FE4FB40205E04280
:1069B2009C8004E0F4529C90FE4FE0F4529B2290A3
:1069C200FE50E0FF700790FE4FE0429722EF90FCEE
:1069D20026B4021212999DFEEF4EFF90FC261299E8
:1069E2008EE05F42972212999DF4FEEF5E90FC26A4
:1069F200F0EE52972290FE4EE0FF24FA60331460CC
:106A02004214606124036003026AAD90FE50E0FE0E
:106A1200700790FE4FE0429B22EE90FE4FB40205BB
:106A2200E0429C8004E0F4529C90FE4FE0F4529BC2
:106A32002290FE50E090FE4F7004E0429422E0F477
:106A420052942290FE50E0701574272F129995C02F
:106A520083C08212999DFEEF4ED082D083F01299AC
:106A62008FE0F595221299EF701312998FC083C0AF
:106A7200821299BFEE4DD082D083F08028EF90FC35
:106A820022B4020E12999D90FC221299871299FA51
:106A9200801312999DC454F0F4FEEF5E90FC221212
:0C6AA200998EE05EF012998FE0F5AD22B5
:10ACFA00EF24FA601114601214601314601424040F
:10AD0A007013E4F5A12275A1012275A1022275A191
:06AD1A00032275A10422D2
:10936B00AB05AA07EA14601914601B14601D146086
:10937B001F24FA6020146022240B7023E5805BFF0E
:10938B0022E5905BFF22E5A05BFF22E5B05BFF22AD
:10939B00E5F25BFF22E58A5BFF22E5C15BFF221250
:1093AB0099B77032EA24FB24FB500624FE600C8034
:1093BB0047AF0212ACFAE59A5BFF22E58F5470FAC5
:1093CB00758F7090FC25E591F0E4F58FE04591F0F9
:1093DB008A8FE05BFF22EA24FA600F14601114609D
:1093EB001324037013E59A5BFF22E5935BFF22E5E1
:0993FB00955BFF22E5AD5BFF224A
:10777C0090FE55EFF0A3EDF090FE55E0FF129993BB
:10778C00E04DF0EF14602114603414603B1460423F
:10779C0024FA605414607B240B600302784590FE3D
:1077AC0055129992E0F5802290FE56E0FF90FC2352
:1077BC00E05F42FD90FE55129992E0F5902290FE0A
:1077CC0055129992E0F5A02290FE55129992E0F58F
:1077DC00B02290FE56E0FF90FC24E05F42F390FE56
:1077EC0055129992E0F5F22290FE55E0FF12999312
:1077FC00C083C082E090FE561299C390FC34E05DC9
:10780C00FDEE4DD082D083F074272F129995E0F5C0
:10781C008A2290FE55E0FF129993C083C082129980
:10782C00ABFD90FC35E05DFDEE4DD082D083F07465
:10783C00272F129995E0F5C1221299B7704390FE4B
:10784C00551299D4500724FE60100278E212ACFA5B
:10785C0090FE55129992E0F59A2290FE55E0FF1297
:10786C009993C083C0821299ABFD90FC26E05DFD1C
:10787C00EE4DD082D083F074272F129995E0F591BC
:10788C002290FE55E0FF24FA601414601B14602251
:10789C002403704274272F129995E0F59A2290FEDA
:1078AC0055129992E0F5932290FE55129992E0F5BB
:1078BC00952290FE55E0FF129993C083C082E0FEA2
:1078CC0090FE56E01299DB4DD082D083F074272FB6
:0778DC00129995E0F5AD22C1
:1078E30090FE57EFF0A3EDF090FE57E0FF1299934F
:1078F300E0FEEDF4FDEE5DF0EF146021146035144D
:10790300603C14604324FA6056146077240B6003D0
:107913000279A990FE57129992E0F5802290FE57C2
:10792300129992E0F59090FE58E0FF90FC23E05FFF
:10793300F452FD2290FE57129992E0F5A02290FE98
:1079430057129992E0F5B02290FE57129992E0F502
:10795300F290FE58E0FF90FC24E05FF452F3229093
:10796300FE57E0FF129993E0FEF58A74272F1299D0
:1079730095C083C08290FE58E0C454F0FF90FC345D
:10798300027A3E90FE57E0FF129993E0FEF5C17430
:10799300272F129995C083C08290FE581299B0FF89
:1079A30090FC35027A3E1299B7703E90FE571299B9
:1079B300D4500724FE6010027A4912ACFA90FE57A5
:1079C300129992E0F59A2290FE57E0FF129993E004
:1079D300FEF59174272F129995C083C08290FE58AB
:1079E3001299B0FF90FC26805290FE57E0FF24FAD4
:1079F300601414601B1460222403704A74272F122E
:107A03009995E0F59A2290FE57129992E0F5932208
:107A130090FE57129992E0F5952290FE57E0FF12DF
:107A23009993E0FEF5AD74272F129995C083C08218
:107A330090FE58E0C454F0FF90FC22E05FF4FFEEA8
:077A43005FD082D083F02226
:106AAE0090FE5AEDF090FE59EFF0146044146076AB
:106ABE00147003026B55147003026B7624FA700384
:106ACE00026BAB147003026BFE240B6003026C505E
:106ADE0090FE59E0FF129993C083C0821299A4FDD3
:106AEE00EE6DD082D083F074272F129995E0F58049
:106AFE002290FE59E0FF1299931299A4FDF4FCEE38
:106B0E005CF59090FC23E05D62FD74272F12999541
:106B1E00C083C0821299E7D082D083F090FE5912C2
:106B2E009992E0F5902290FE59E0FF129993C0835E
:106B3E00C0821299A4FDEE6DD082D083F074272FFF
:106B4E00129995E0F5A02290FE59E0FF129993C09C
:106B5E0083C0821299A4FDEE6DD082D083F074278B
:106B6E002F129995E0F5B02290FE59E0FF129993FD
:106B7E001299A4FDF4FCEE5CF5F290FC24E05D624B
:106B8E00F374272F129995C083C0821299E7D08291
:106B9E00D083F090FE59129992E0F5F22290FE59B0
:106BAE00E0FF1299931299A4F4FDEE5DF58A742715
:106BBE002F129995C083C08290FE5AE0C454F0FF04
:106BCE0090FC34E05FFFEE6FD082D083F090FE59E0
:106BDE00E0FF129993C083C0821299A4540FFDEE68
:106BEE006DD082D083F074272F129995E0F58A220A
:106BFE0090FE59E0FF1299931299A4F4FDEE5DF503
:106C0E00C174272F129995C083C08290FE5A129993
:106C1E00B0FF90FC35E05FFFEE6FD082D083F09036
:106C2E00FE59E0FF129993C083C0821299A4541C9E
:106C3E00FDEE6DD082D083F074272F129995E0F57A
:106C4E00C1221299B7706890FE591299D450072438
:106C5E00FE6027026D6612ACFA90FE59E0FF1299A3
:106C6E0093C083C0821299A4FDEE6DD082D083F0C2
:106C7E0074272F129995E0F59A2290FE59E0FF1293
:106C8E0099931299A4FDF4FCEE5CF59190FC26E02C
:106C9E005D629774272F129995C083C0821299E76F
:106CAE00D082D083F090FE59129992E0F591229005
:106CBE00FE59E0FF24FA602B146046146061240331
:106CCE006003026D6690FE59E0FE129993C083C078
:106CDE00821299CAD082D083F074272E129995E031
:106CEE00F59A2290FE59E0FE129993C083C082124B
:106CFE0099CAD082D083F074272E129995E0F5931D
:106D0E002290FE59E0FE129993C083C0821299CA56
:106D1E00D082D083F074272E129995E0F5952274C7
:106D2E00272F129995C083C0821299A41299DB6DF8
:106D3E00D082D083F074272F129995C083C082E041
:106D4E00FF90FE5AE0540FFEEF6ED082D083F0908B
:096D5E00FE59129992E0F5AD22F4
:10AF6D00786DE6FF90FF8093FE74802FF582E434B8
:08AF7D00FFF583EEF006E62269
:10AFB400C3EE940240037FFF2274002FF58274EEE7
:07AFC4003EF583E493FF2238
:10A2C70090FE5BEEF0A3EFF0C3EE94025040748073
:10A2D7006480700374FFF4703530AF02D230C2AFC0
:10A2E70090FE5CE0240090FE5BE034EEF5F9A3E01D
:10A2F700F5FA786D764012AF6DB480FAAF05786DD8
:0FA30700A6077B01796D12FFC0303002D2AF2262
:10ABBC0074806480700374FFF4701E30AF02D23066
:10ABCC00C2AF75F9EEE4F5FA786DF612AF6DB440DC
:0AABDC00FA12FF80303002D2AF22DF
:0C8CED00C13141FDCA0043FDCB00000076
:10AF070090FDCBE0FBA3E0FAA3E0F9EA494B2290DE
:0CAF1700FDCBA3E0FAA3E0F5828A8322C0
:10A7910075A101E5A1B4011BEF24FE600C14600E4C
:10A7A1002403702375A49C801E75A4DC801975A4F4
:10A7B100FC801443F580EF24FE60092402700875C3
:0AA7C100A4B8800375A4F8D2BD22ED
:0CB1480090FDCBEBF0A3EAF0A3E9F022AD
:10AC860030310CEF70037F862290FDCAE0FF2275FB
:10AC9600A101E5A1B40107EF04F5A6AFA722EF7065
:07ACA60003AFA622AFA722B5
:03006B00029C7B79
:109C7B00C0E0C0F0C083C082C0D075D000C000C0AF
:109C8B0001C002C003C004C005C006C007C23175C5
:109C9B00A101E5A164017019F5A612AF07602AE5D1
:109CAB00A530E6047F0180027F0012AF16ADA780BE
:109CBB001512AF076013E5A530E6047F0180027F24
:109CCB000012AF167D10121ECC43A580D007D00614
:109CDB00D005D004D003D002D001D000D0D0D08298
:079CEB00D083D0F0D0E0327D
:068CF90041FE6301C132DF
:06B1B10090FE63EFF022A6
:10AF8500EF6005D232758680E5FFB430037F01227C
:08AF950075FF30D2AF7F0022EE
:08B19B00303204D2AED2BE2214
:105A0700444247434D4420537472696E6720427580
:105A1700666665722046756C6C0D0A002573202535
:105A270058202558202558202558006275730044B2
:105A37004247434D44206275733A204275733D30A7
:105A47007825302E32582C20506F72743D307825CF
:105A5700302E32582C2053706565643D30782530E0
:105A67002E32580D0A0063697200444247434D4481
:105A7700206369723A20436F64653D307825302E84
:105A870032580D0A0077723000444247434D442094
:105A97007772303A2049443D307825302E32582CE1
:105AA700205265673D307825302E32582C204461CE
:105AB70074613D307825302E32580D0A00726430FB
:105AC70000444247434D44207264303A2049443DE4
:105AD700307825302E32582C205265673D30782596
:105AE700302E32582C20446174613D0030782530C7
:105AF7002E32580D0A0074623000444247434D4429
:105B0700207462303A2049443D307825302E32588F
:105B17002C205265673D307825302E32582C204D89
:105B270061736B3D307825302E32582C20446174D8
:105B3700613D0063623000444247434D4420636245
:105B4700303A2049443D307825302E32582C2052A7
:105B570065673D307825302E32582C204D61736BA8
:105B67003D307825302E32582C20446174613D0039
:105B770077723100444247434D44207772313A20CF
:105B870049443D307825302E32582C205265673DE8
:105B9700307825302E32582C20446174613D30789E
:105BA70025302E32580D0A007264310044424743B3
:105BB7004D44207264313A2049443D307825302ED7
:105BC70032582C205265673D307825302E32582CBC
:105BD7002053697A653D307825302E32582C204481
:105BE7006174613D002852656164206E756D626560
:105BF70072206578636565642061206D6178206F28
:105C07006620256420627974657329000D0A0020D7
:105C170000307825302E32582C2000746231004431
:105C27004247434D44207462313A2049443D30781D
:105C370025302E32582C205265673D307825302E7E
:105C470032582C204D61736B3D307825302E3258F9
:105C57002C20446174613D00636231004442474334
:105C67004D44206362313A2049443D307825302E37
:105C770032582C205265673D307825302E32582C0B
:105C8700204D61736B3D307825302E32582C2044DF
:105C97006174613D0077723200444247434D4420AE
:105CA7007772323A2049443D307825302E32582CCD
:105CB700205265673D307825302E34582C204461BA
:105CC70074613D307825302E32580D0A00726432E7
:105CD70000444247434D44207264323A2049443DD0
:105CE700307825302E32582C205265673D30782584
:105CF700302E34582C2053697A653D307825302E64
:105D070032582C20446174613D0074623200444271
:105D170047434D44207462323A2049443D30782548
:105D2700302E32582C205265673D307825302E347E
:105D3700582C204D61736B3D307825302E32582C0E
:105D470020446174613D0063623200444247434D21
:105D570044206362323A2049443D307825302E3260
:105D6700582C205265673D307825302E34582C202A
:105D77004D61736B3D307825302E32582C204461AD
:105D870074613D004552524F523A204949432066BB
:105D970061696C65642025642C204949434164642A
:105DA700723D307825302E32582C20526567416479
:0D5DB70064723D307825302E32580D0A0000
:088CFF0041FC010041FBFF00F4
:1074140078ED7CFB7D017BFF122087EF2278ED7CE9
:10742400FB7D017BFF122087EF22A3F090FBE6E0B7
:10743400FF90FBE9E0FCA3E090FCD0FD7B017AFB2C
:1074440079EDE4F0A304F02278ED7CFB7D017BFF71
:10745400122087EF2278ED7CFB7D017BFF122087D1
:10746400EF227BFF7A5C791890FC03E024EDF5822F
:10747400E434FBF583E0FFE490FB39F0A3EFF02262
:1074840078ED7CFB7D017BFF122087EF2290FBEDE2
:10749400F090FBE6E0FF90FBE8E0FD7B017AFB79EE
:1074A400ED2278ED7CFB7D017BFF122087EF22909B
:1074B400FBE8E0FEA3E04EF0A3E0F022E4F0A374C6
:1074C40012F07BFF7A5B79EC90FB39E4F0A3741241
:1074D400F0227BFF7A5A79F390FBEDE0FF90FB39C1
:1074E400E422F0A3EDF0A3EBF0A3EAF0A3E9F0901B
:1074F400FC02E4F0A3740AF0E4A3F0A3F02290FBEE
:10750400E8E0FD90FBEAE0FB22FDE0FBA3E0FAA348
:10751400E0F9A3E0FFA3E090FC5ACFF0A3EFF0ED75
:1075240022A3F0A37401F0A322A3F0A37422F043D6
:10753400FF407AFF7980121EC853FFBF22E0FEA3EA
:10754400E0FF90FC02E0FCA3E0FDC39FEC9E22E080
:10755400FFE490FB3BF0A3EFF022D390FC03E09414
:107564000090FC02E0940022C390FC05E094039098
:10757400FC04E09400227BFF90FBE5E0FFA3E02203
:1075840078ED7CFB7D017BFF122087EF22E054FE27
:10759400FD7B0190FC5AE4F0A322A3E024FDF090CB
:1075A400FC02E034FFF02290FC5CEFF090FBFFE083
:1075B400FF227BFF7A5C79132290FBEDE0FF90FBC6
:0D75C400EAE02290FBEDE0FF90FBECE022FE
:103CE50012AC5F90FE64EFF0F470030240A8E0FFB1
:103CF50090FC01E0FE04F074ED2EF582E434FBF552
:103D050083EFF090FC01E0D39412400E7BFF7A5ACA
:103D1500790712A3B1E490FC01F090FE64E0FF6422
:103D25000A6008EF640D60030240A8E490FC01F00E
:103D350090FB6774FFF0A3745AF074231275257411
:103D4500FFF0748012752574FBF0A374E5127526D7
:103D550074FBF0A374E712752674FBF0A374E912E3
:103D6500752674FBF0A374EBF012749F126539E4A9
:103D750090FBF0F07A5A7932127414701D7A5A79E0
:103D8500361240AE90FBE6E0FF12750212A8A59030
:103D9500FBE6E090FBFFF00240A87A5A796D1274B9
:103DA50014703F7A5A797112757ACF12747C12A306
:103DB500B1D23190FBE6E090FDCAF090FDCBE0FB7F
:103DC500A3E0FAA3E0F9EA494B70030240A890FD8D
:103DD500CBA3A3E0F5828A837D10E4FF121ECC02FB
:103DE50040A87A5A798C12742170127A5A799012F5
:103DF50040AE1275027F7512B10B0240A87A5A794E
:103E0500C412742170207A5A79C812757A90FB39D8
:103E1500CFF0A3EFF090FBE7E0FFA3E0CF127556DC
:103E250012A3B1023E5D7A5A79FD12744C70117A73
:103E35005B79011240E11275027F6312B10B8018A4
:103E45007A5B793A12744C70337A5B793E1240E1B1
:103E55001275027F5312B10B90FBE8E0FF12B06DB3
:103E650090FBEBE4F0A3EFF07BFF7A5A79F390FB3C
:103E7500EBE0FFA3E090FB39CF0240697A5B7977ED
:103E850012745970247A5B797B12411490FBEAE035
:103E950090FBEDF090FBE6E0FF90FBE8E090FD1075
:103EA50012743F12949B0240A87A5B79AF12745941
:103EB50070777A5B79B3124114D390FBEAE09412E0
:103EC50090FBE9E0940040061274C012A3B190FB88
:103ED500E6E04401FFC00712749AA3E0FFA3E09057
:103EE500FD10CFF0A3EFF0D00712949BEF60030213
:103EF50040A890FC02F0A3F090FBE9127541502612
:103F0500ED540F70061275B612A3B190FC03E05480
:103F150007700312422412746612422E70DA90FC66
:103F250002E004F080D20240387A5C79221274846F
:103F350070277A5C79261241CA12949BEF600302BE
:103F450040A81275BDFEEF6E127491124217600300
:103F55000240A81274D60240697A5C795F127484B3
:103F650070287A5C79631241CA12949BEF60030250
:103F750040A81275BDF4FEEF5E12749112421760EF
:103F8500030240A81274D60240697A5C799C1274C7
:103F9500A670171274B37A5C79A012414790FBECB6
:103FA500E012742E1291970240A87A5C79D41274AB
:103FB500A6600302403E1274B37A5C79D812414779
:103FC500D390FBECE0941290FBEBE09400400612DA
:103FD50074C012A3B190FBE6E04401FFC00790FB5B
:103FE500E9E0FCA312749DA3E0FFA3E090FCD0CF11
:103FF500F0A3EFF0D007129197EF60030240A8906D
:10400500FC02F0A3F090FBEB1275415026ED540F26
:1040150070061275B612A3B190FC03E05407700345
:1040250012422412746612422E70DA90FC02E004E9
:10403500F080D21275B60240A57A5D7911127584A9
:1040450070291274B37A5D791512417A129197EF3E
:1040550070511275C7FEEF6E12742E129197EF70A4
:10406500421274D6F0A3EFF00240A57A5D794E12A4
:104075007584702F1274B37A5D795212417A129158
:1040850097EF701F1275C7F4FEEF5E12742E129132
:1040950097EF700F7BFF7A5A79F390FBED127479E5
:1040A50012A3B190FE64E0FF227BFF90FBE5E0FFE9
:1040B500A3E090FB39CFF0A3EFF090FBE7E0FFA37F
:1040C500E090FB3BCFF0A3EFF090FBE9E0FFA3E02E
:1040D50090FB3DCFF0A3EFF012A3B1227BFF90FB45
:1040E500E5E0FFA3E090FB39CFF0A3EFF090FBE70D
:1040F500E0FFA3E090FB3BCFF0A3EFF090FBE9E0FE
:10410500FFA3E090FB3DCFF0A3EFF012A3B1227B1C
:10411500FF90FBE5E0FFA3E090FB39CFF0A3EFF0C4
:1041250090FBE7E0FFA3E090FB3BCFF0A3EFF0901F
:10413500FBE9E0FFA3E090FB3DCFF0A3EFF012A376
:10414500B1227BFF90FBE5E0FFA3E090FB39CFF0C8
:10415500A3EFF090FBE9E0FFA3E090FB3BCFF0A3DA
:10416500EFF090FBEBE0FFA3E090FB3DCFF0A3EF7A
:10417500F012A3B1227BFF90FBE5E0FFA3E090FBEB
:1041850039CFF0A3EFF090FBE9E0FFA3E090FB3B14
:10419500CFF0A3EFF090FBEBE0FFA3E090FB3DCF6A
:1041A500F0A3EFF012A3B190FBE6E04401FF90FB12
:1041B500E9E0FCA3E0FD7B017AFB79ED90FCD0E41E
:1041C500F0A304F0227BFF90FBE5E0FFA3E090FB6A
:1041D50039CFF0A3EFF090FBE7E0FFA3E090FB3BC6
:1041E500CFF0A3EFF090FBE9E0FFA3E090FB3DCF1C
:1041F500F0A3EFF012A3B190FBE6E04401FF90FBC2
:10420500E8E0FD7B017AFB79ED90FD10E4F0A30475
:10421500F02290FD10E4F0A304F012949BEF227BB2
:10422500FF7A5C791612A3B12212A3B190FC03E0C8
:0342350004F02270
:10949B0090FD0BEF1274E690FBFFE0FF90FD0B7A53
:1094AB00FD790C12759104F0A3F01275D190FC00AC
:1094BB00EFF0E0FEC00690FD0BE090FD0D12750D78
:1094CB0030E0047F0080027F021275AB1275D1D0A1
:1094DB00E04F90FC00F0602390FC03E0FF12B124FE
:1094EB0012755E400312759E90FC05E004F0700649
:1094FB0090FC04E004F012756C409C90FC00E0FFC3
:10950B00601F7BFF7A5D798B12747B90FD0B12755C
:10951B005390FD0CE0FF90FB3DE4F0A3EFF012A3A2
:07952B00B190FC00E0FF22FB
:1091970090FCCAEFF0A3EC1274E690FBFFE0FF909F
:1091A700FCCA7AFC79CB1275917402F0A314F01201
:1091B70075D190FC00EFF0E0FEC00690FCCAE0908D
:1091C700FCCD12750D30E0047F0080027F0212751E
:1091D700AB1275D1D0E04F90FC00F0602390FC03F8
:1091E700E0FF12B12412755E400312759E90FC05D4
:1091F700E004F0700690FC04E004F012756C409AED
:1092070090FC00E0FF60217BFF7A5D798B12747B15
:1092170090FCCA12755390FCCBE0FFA3E090FB3D96
:0E922700CFF0A3EFF012A3B190FC00E0FF2205
:10B06D0090FF807485F0A3EFF0746E12752D786EDD
:03B07D00E6FF22C9
:0DB10B0090FF80EFF0A3EDF0EB12752D2208
:0E8D070043F9FB01FA0541F9FF0041F9FE00B6
:1083CA0090FD79E0FBA3E0FAA3E0F92290001FE414
:1083DA00F5F0121B6890001502194BE0FEA3E0FFAE
:1083EA007C007D051219CE90F9FBE0FBA3E0FAA30D
:1083FA00E02FF9EA3EA801FCAD037B017AFF798000
:10840A002290001FE4F5F0121B68900016021E1954
:10841A0090F9FFE0FFC390FA04E09F7480F890FAA5
:10842A0003E06480982290001FE475F001121ACFCD
:10843A00FEC3E5F02290F9FFE075F005A4FF90F97C
:10844A00FBE0FBA3E0FAA3E022EBF0A3EAF0A3E946
:10845A00F022FD7401F0A374FFF0A37480F022905F
:10846A00000402194B7E007F0512190C90F9FFE0F7
:10847A0004F0227F057E0012222AEF2290F9FFE003
:10848A004480F02290001FE4F5F0021B682404F9EE
:06849A00E43AFA02193277
:1047880090FD79128453900006121E1990FD7C1238
:1047980084531283CA12193224F9B4070040030261
:1047A8004CB89047B875F003A4C58325F0C583734A
:1047B8000247CD024894024A47024A9D024AF6023D
:1047C8004B70024C0C90FD7C1283CD12846930E151
:1047D800751283CA128414C003C002C0011283CAAE
:1047E8001283DFFDD001D002D00312AD881283CA34
:1047F8001284309432EE94005003024CB81283D6DF
:10480800FF128404128BABEF602A1283CA128469E8
:1048180030E019128414C003C002C0011283CA1206
:1048280083DFFDD001D002D00312ADEB1283CA742E
:1048380008024CB51283CA1283DFFFE4FD12ABE60F
:1048480090FD79024A811283CA12846930E01912F4
:104858008414C003C002C0011283CA1283DFFDD0D2
:1048680001D002D00312ADEB1283CA128414C00324
:10487800C002C0011283CA1283DFFDD001D002D06A
:104888000312ADA91283CA7405024CB51283CA1269
:1048980083DFFFE4FD12ABE61283CA1283DF124CFA
:1048A800B990FD7930E61E1283CD128414C003C07E
:1048B80002C0011283CA1283DFFDD001D002D003E7
:1048C80012AE0C801C1283CD128414C003C002C027
:1048D800011283CA1283DFFDD001D002D00312AEC9
:1048E8002DE490FF88F012A3FE7C017D00121A359A
:1048F80090FF88E02480F582E434FFF583EDF090A2
:10490800FF88E004F0E0C3940840DB1283CA1284F5
:1049180014C003C002C0011283CA1283DF90FCE5F1
:1049280012845CD001D002D00312AA651283CA1285
:1049380083DFFF1284041201D91283CA128414C0BF
:1049480003C002C0011283CA1283DF90FCEC1284F8
:104958005CD001D002D003128E72EF70241283CA89
:10496800128414C003C002C0011283CA1283DFFD7F
:10497800D001D002D00312AE8E1283CA7407024C43
:10498800B51283CA1283DFFF12840412AC38128373
:10499800CA1283DFFF128404128BABEF70241283D8
:1049A800CA128414C003C002C0011283CA1283DF72
:1049B800FDD001D002D00312AE8E1283CA74070252
:1049C8004CB51283CA128414C003C002C0011283FA
:1049D800CA1283DFFD90FCF312845DD001D002D0AF
:1049E8000312AA911283CA900019121E19E94A4BA0
:1049F800704590F9FFE0C394085039E490FA03F049
:104A0800A3F012841A50181283E512847D60109066
:104A1800FA04E004F070EB90FA03E004F080E3128B
:104A2800841A401312843F2FF9EA35F01283FF12DB
:104A3800846F80031284861283CA7409024CB512EB
:104A480083CA1284309407EE94005003024CB812C3
:104A58008414C003C002C0011283CA1283DFFDD0D0
:104A680001D002D00312AB3EEF90FD79600B1283A8
:104A7800CD12848E740A024CB51283CD128414C0F0
:104A880003C002C0011283CA1283DFFDD001D00225
:104A9800D00302AE8E1283CA129E2DEF703112839C
:104AA800CA128430940AEE94005003024CB812845F
:104AB8000BC003C002C0011283CA1283DFFDD001FC
:104AC800D002D00312AE8E1283CA7407024CB512FC
:104AD80083CA1283D6124CB990FD7930E608128346
:104AE800CD740D024CB51283CD740B024CB5E49015
:104AF800FF80F01283CA12841412B0E2EF700C9097
:104B0800FF80E004F0E0C394FA40E8E490FF81F00D
:104B18001283CA12841412B0E2BF010C90FF81E024
:104B280004F0E0C394FA40E81283CA128414C00364
:104B3800C002C0011283CA1283DFFDD001D002D0A7
:104B48000312ADCA1283CA128414C003C002C00182
:104B58001283CA1283DFFDD001D002D00312ADA99F
:104B68001283CA740C024CB590FD7C1283CD12845A
:104B78006930E16C1283CA128430944BEE94005071
:104B880003024CB812848E129E2DEF70451283CA10
:104B980012846930E221128414C003C002C00112D9
:104BA80083CA1283DFFDD001D002D00312AE6E1289
:104BB80083CA7407024CB590FD7912844B1284970E
:104BC800440412199A1283CA90001FE475F0320245
:104BD8001B6890FD7912844B12849754FB024CB5E4
:104BE8001283CA128414C003C002C0011283CA12FD
:104BF80083DFFDD001D002D00312AE6E1283CA74D7
:104C080007024CB51283CA1283DFFF12AEAE90FAC8
:104C180000EFF030E56C1283CA1283D6FF128404C9
:104C280012A7CB90FF80E0FD20E71CA3E0FF20E364
:104C3800161283CA90FCD6EFF0127BAAEF602012FE
:104C480083CA740B024CB590FF80E030E7031284EE
:104C58008690FF81E030E30790F9FEE04408F01207
:104C680083CA128414C003C002C0011283CA12830B
:104C7800DFFDD001D002D00312AE8E1283CA7407B2
:104C8800802B1283CA12843094FAEE9400402112C9
:104C9800840BC003C002C0011283CA1283DFFDD097
:104CA80001D002D00312AE8E1283CA740712199A69
:0B4CB80022FF12AEAE90FA00EFF022D7
:109E2D0090FD12128453128414C003C002C001901D
:109E3D00FD121283CD1283DFFD90FCFA7401F0A3A5
:109E4D0074FDF0A37415F0D001D002D00312A495C7
:109E5D00EF7002FF2290FD121283CD1283DFFF7B84
:109E6D00017AFD7917129EFAEF7002FF2290FD170D
:109E7D00E0FEA3E0FF90FD15E0B50608A3E0B507F1
:079E8D00037F01227F002288
:107BAA0090FCD2128453A3EDF0A3E0540FFF90F996
:107BBA00FEE0FEEFD39E40028002AF0690F9FEEF90
:107BCA00F012A6A2E490FA01F0A3F090FCD5E0FF2F
:107BDA0090FA01E0FCA3E0FDC39F7480F8EC648096
:107BEA00984003027C7090FCD21283CD1283DFFF8F
:107BFA0012840490FD41EDF090FCD5E090FD42F036
:107C0A00127E41EF7002FF2290F9FFE0C394085000
:107C1A0039E490FA03F0A3F012841A50181283E59B
:107C2A0012847D601090FA04E004F070EB90FA037D
:107C3A00E004F080E312841A401312843F2FF9EA19
:107C4A0035F01283FF12846F800312848612840433
:107C5A007D05128DCB90FA02E004F0700690FA01CD
:107C6A00E004F0027BD590FCD5E0701890FCD212AB
:107C7A0083CD1283DFFF128404E490FD41F0A30454
:107C8A00F0127E4190FCD5E090FF80F090FCD6E0A7
:107C9A0090FF81F090FCD21283CD128414C003C0ED
:107CAA0002C00190FCD21283CD1283DFFD90FD0148
:107CBA007401F0A374FFF0A37482F0D001D002D053
:107CCA000312AB681284047D0A128DCB128135909F
:107CDA00FCD712845390FCD21283CD1283DFFF1299
:107CEA00840412A80290FCD712844BF8AC021284C6
:0E7CFA00027F1412847F60037F00227F01222C
:068D150043FB1C01FFC03E
:1085710090FB2AE0FCA3E0FDA3E0FEA3E0FF90FB5B
:1085810026E0F8A3E0F9A3E0FAA3E022121DDC90B3
:10859100FC81E0FCA3E0FDA3E0FEA3E0FF227E005E
:1085A1007F407D0090FB1CE0FBA3E0FAA3E022EBFF
:1085B1002FFFEA3EFEE93DFDE83CFC22F9A3E05431
:1085C1000F75F004A4F58285F08322EF4BFFEE4A8C
:1085D100FEED49FDEC48FC226FFFEA6EFEE96DFD00
:1085E100E86CFC225FFFEA5EFEE95DFDE85CFC22CF
:1085F10090FC7DC9F0A3EAF0A3E9F07B017AFB7955
:108601000522EF6BFFEE6AFEED69FDEC68FC22903E
:10861100FC81021DDC121D4990FC7A22F074072BAB
:10862100F58274FB3AF5832274062BF58274FB3ACA
:0D863100F58322F912224EE490FB19F0228D
:10A6A20090FB05121DE86745230190FB09121DE886
:10A6B200EFCDAB8990FB0D121DE898BADCFE90FB42
:10A6C20011121DE81032547690FB15121DE8C3D208
:0DA6D200E1F012859F128634A3F0A3F02260
:108DCB0090FDCEEBF0A3EAF0A3E9F0A3EDF0FF905A
:108DDB00FB1BE02FF090FB1AE03400F090FDD1E08C
:108DEB00FF7003028E7190FB19E0FEC374409EFE70
:108DFB00C39F5004AF06800590FDD1E0FF90FB1F91
:108E0B00EFF07E001285A5F990FB19E0FD7C00E9DF
:108E1B002DF9EC3AA801FCAD0390FDCE1285A8F913
:108E2B0012190C90FB1FE0FF90FB19E02FF090FD47
:108E3B00CFE48FF0121A6B90FDD1E0FF90FB1FE097
:108E4B00FEC3EF9E90FDD1F090FB19E0C394404020
:108E5B008B90FB1C1285851285F1125DC412859FC8
:078E6B00128634028DE7229C
:108135001285A5F990FB19E0FF04F08F8275830085
:1081450074801219AC90FB19E0FFC374409FC3946F
:1081550002500712859FF912224E90FB1AE0FEA3EA
:10816500E07803C333CE33CED8F9F0EE90FB1AF0A6
:10817500E0FF1285A5F990003EEF1219AC90FB1BAC
:10818500E090003F1219AC90FB1C1285851285F119
:10819500125DC4E490FB20F0A3F0C390FB21E094B2
:1081A5001490FB20E0648094805066E0FEA3E0FF1D
:1081B5002405F58274FB3EF583E0FD90FF80F074A5
:1081C500082FF58274FB3EF583E0FF90FB20E0FA73
:1081D500A3E0FB2405F58274FB3AF583EFF0740800
:1081E5002BF58274FB3AF583EDF0128629E0FF90BA
:1081F500FF8012861DE0FE128629EE12861DEFF025
:1082050090FB21E02404F090FB20E03400F0028193
:058215009F1285FC2210
:105DC40090FC7AEBF0A3EAF0A3E9F0121CF990FB43
:105DD40022121DDC900004121D1990FB26121DDCFA
:105DE400900008121D1990FB2A121DDC90000C1261
:105DF4001D1990FB2E121DDC900010121D1990FB32
:105E040032121DDCE490FC80F090FC80E0FFD3941F
:105E14004F40030260B0EFC394105003025EAC9095
:105E2400FC7D1285A8F9A3E024081285C0121D196F
:105E3400C00790FC7DA3A3A3E0240D1285C0121D0E
:105E4400A0D007EB1285D9C00790FC7D1285A8F974
:105E5400A3E024021285C0121DA0D007128603C03D
:105E64000790FC7D1285A81285BD121DA0D00712D3
:105E7400860390FC8112858D7801121CE6C004C053
:105E840005C006C007128590781F121CBFD003D02E
:105E940002D001D0001285CCC00790FC7D1285A8E9
:105EA4001285BDD007121D6390FC7D1285A8128552
:105EB400BD121D1912861090FC81128582FBC00050
:105EC400C001C002C00390FB221285937805121C06
:105ED400E6C004C005C006C00790FB221285937873
:105EE4001B121CBFD003D002D001D0001285CCD02D
:105EF40003D002D001D0001285B012861090FC802D
:105F0400E0D394135048A3128582FBC000C001C0A3
:105F140002C00390FB26128593121CB290FB2E1232
:105F240085821285E5C004C005C006AB07128571E1
:105F34001285E5D002D001D0001285CCEF2499FF60
:105F4400EE3479FEED3482FDEC345A02602E90FC7E
:105F540080E0D39427502EA3128582FBC000C00199
:105F6400C002C0031285711285D990FB2E1285825E
:105F74001285D9EF24A1FFEE34EBFEED34D9FDEC0C
:105F8400346E02602E90FC80E0D3943B506FA312D9
:105F94008582FBC000C001C002C00390FB2E1285A5
:105FA400741285E5C004C005C006AB07A31285932F
:105FB40090FB26A3A3A3E01285E5D002D001D00074
:105FC4001285CCC004C005C006AB0790FB2E128519
:105FD4009390FB2A1285821285E5D002D001D0006D
:105FE400EB4FFFEA4EFEE94DFDE84CFCEF24DCFFED
:105FF400EE34BCFEED341BFDEC348F802D90FC811F
:10600400128582FBC000C001C002C0031285711258
:1060140085D990FB2E1285821285D9EF24D6FFEE06
:1060240034C1FEED3462FDEC34CAFCD003D002D09E
:1060340001D0001285B012861012859090FB3212A6
:106044008582FBEF2BFFEE3AFEED39FDEC38FC12B6
:10605400861090FB2E128593A3121DDC90FB2A124E
:106064008593A3121DDC90FB26128593781E121CC7
:10607400E6C004C005C006C00790FB2612859378CD
:1060840002121CBFD003D002D001D0001285CCA3D1
:10609400121DDC90FB22128593A312858D90FB22A6
:1060A400121DDC90FC80E004F0025E0D90FC7A127C
:1060B40085A8F9C002C001121CF990FB2212858246
:1060C4001285B1D001D0021286161285A82404F9D3
:1060D400E43AFAC002C001121CF912857F1285B19C
:1060E400D001D0021286161285A82408F9E43AFADF
:1060F400C002C001121CF990FB2A1285821285B1DC
:10610400D001D0021286161285A8240CF9E43AFABA
:10611400C002C001121CF990FB2E1285821285B1B7
:10612400D001D0021286161285A82410F9E43AFA96
:10613400C002C001121CF990FB321285821285B193
:07614400D001D002021D4949
:030000000296DD88
:0C96DD00787FE4F6D8FD75816E029724BA
:10183C00E709F608DFFA8046E709F208DFFA803E8E
:10184C0088828C83E709F0A3DFFA8032E309F6087B
:10185C00DFFA8078E309F208DFFA807088828C83E3
:10186C00E309F0A3DFFA806489828A83E0A3F60897
:10187C00DFFA805889828A83E0A3F208DFFA804C71
:10188C0080D280FA80C680D4806980F28033801048
:10189C0080A680EA809A80A880DA80E280CA8033B1
:1018AC0089828A83ECFAE493A3C8C582C8CCC58329
:1018BC00CCF0A3C8C582C8CCC583CCDFE9DEE780F9
:1018CC000D89828A83E493A3F608DFF9ECFAA9F078
:1018DC00EDFB2289828A83ECFAE0A3C8C582C8CCCE
:1018EC00C583CCF0A3C8C582C8CCC583CCDFEADEE7
:1018FC00E880DB89828A83E493A3F208DFF980CC49
:10190C0088F0EF60010E4E60C388F0ED2402B40441
:10191C000050B9F582EB2402B4040050AF232345E8
:06192C00822390188C7369
:10193200BB010689828A83E0225002E722BBFE02B3
:09194200E32289828A83E49322E6
:10194B00BB010CE58229F582E5833AF583E0225051
:10195B0006E92582F8E622BBFE06E92582F8E2229B
:0D196B00E58229F582E5833AF583E49322B5
:10197800BB010989828A83F8E028F022500327F7FF
:1019880022BBFE05F8E328F3228A838982F8E493D0
:02199800282203
:10199A00BB010689828A83F0225002F722BBFE012C
:0219AA00F32226
:1019AC00F8BB010DE58229F582E5833AF583E8F071
:1019BC00225006E92582C8F622BBFE05E92582C81D
:0219CC00F22205
:1019CE00EF8DF0A4A8F0CF8CF0A428CE8DF0A42E2D
:0219DE00FE22E7
:1019E000BC000BBE0029EF8DF084FFADF022E4CCEB
:1019F000F875F008EF2FFFEE33FEEC33FCEE9DECB4
:101A0000984005FCEE9DFE0FD5F0E9E4CEFD22EDF9
:101A1000F8F5F0EE8420D21CFEADF075F008EF2F43
:101A2000FFED33FD4007985006D5F0F222C398FD34
:051A30000FD5F0EA22D1
:101A3500C2D5EC30E709B2D5E4C39DFDE49CFCEECC
:101A450030E715B2D5E4C39FFFE49EFE1219E0C34B
:101A5500E49DFDE49CFC80031219E030D507C3E446
:061A65009FFFE49EFE223B
:101A6B00C5F0F8A3E028F0C5F0F8E5821582700206
:061A7B001583E038F022A3
:101A8100A3F8E0C5F025F0F0E58215827002158318
:061A9100E0C838F0E82275
:101A9700BB0110E58229F582E5833AF583E0F5F08D
:101AA700A3E0225009E92582F886F008E622BBFE6A
:101AB7000AE92582F8E2F5F008E222E5832AF583B0
:081AC700E993F5F0A3E9932275
:101ACF00BB010FF8E58229F582E5833AF583E80239
:101ADF001A815011C58229F808C5F026C6F5F018ED
:101AEF00C58236C622BBFE15C58229F808E2C5F0AD
:101AFF0025F0F218E2C5823582F2E58222E5832ACB
:0C1B0F00F583E993F5F0A3E993C5F022FB
:101B1B00BB010DC58229C582C5833AC583021A6BE9
:101B2B005011C58229F808E5F026F618F5F0E58284
:101B3B0036F622BBFE11C58229F808E225F0F5F036
:101B4B00F218E23582F222F8E58229F582E5832A42
:0D1B5B00F58374019325F0F5F0E493382232
:101B6800F8BB0111E58229F582E5833AF583E8F0AF
:101B7800E5F0A3F0225009E92582C8F608A6F0226C
:0D1B8800BBFE09E92582C8F2E5F008F22253
:101B9500E88FF0A4CC8BF0A42CFCE98EF0A42CFCEF
:101BA5008AF0EDA42CFCEA8EF0A4CDA8F08BF0A46D
:101BB5002DCC3825F0FDE98FF0A42CCD35F0FCEBCC
:101BC5008EF0A4FEA9F0EB8FF0A4CFC5F02ECD3991
:0F1BD500FEE43CFCEAA42DCE35F0FDE43CFC22FE
:101BE40075F008758200EF2FFFEE33FECD33CDCCB8
:101BF40033CCC58233C5829BED9AEC99E58298403B
:101C04000CF582EE9BFEED9AFDEC99FC0FD5F0D617
:101C1400E4CEFBE4CDFAE4CCF9A88222B800C1B941
:101C24000059BA002DEC8BF084CFCECDFCE5F0CB7F
:101C3400F97818EF2FFFEE33FEED33FDEC33FCEBB8
:101C440033FB10D703994004EB99FB0FD8E5E4F973
:101C5400FA227818EF2FFFEE33FEED33FDEC33FC60
:101C6400C933C910D7059BE99A4007EC9BFCE99A54
:101C7400F90FD8E0E4C9FAE4CCFB2275F010EF2F99
:101C8400FFEE33FEED33FDCC33CCC833C810D70799
:101C94009BEC9AE899400AED9BFDEC9AFCE899F8D4
:0E1CA4000FD5F0DAE4CDFBE4CCFAE4C8F92267
:10A52000C2D5E830E70FB2D5E4C39BFBE49AFAE466
:10A5300099F9E498F8EC30E717B2D512A556121C39
:10A5400020E4C39BFBE49AFAE499F9E498F88003C9
:10A55000121C2030D50DE4C39FFFE49EFEE49DFD58
:04A56000E49CFC2259
:0D1CB200CFF4CFCEF4CECDF4CDCCF4CC22C7
:101CBF00E8600FECC313FCED13FDEE13FEEF13FF03
:031CCF00D8F12227
:101CD200E86010ECA2E713FCED13FDEE13FEEF1328
:041CE200FFD8F02215
:101CE600E8600FEFC333FFEE33FEED33FDEC33FC5C
:031CF600D8F12200
:101CF900BB010789828A830222A75005E9F8021DE0
:101D090087BBFE05E9F80222B389828A830222BFD2
:101D1900BB010DE58229F582E5833AF5830222A705
:101D29005007E92582F8021D87BBFE07E92582F8DD
:101D39000222B3E58229F582E5833AF5830222BFBF
:101D4900BB010789828A83021DDC5005E9F8021D5F
:0A1D5900D0BBFE05E9F80222F822D3
:101D6300BB010DE58229F582E5833AF583021DDC8B
:101D73005007E92582F8021DD0BBFE07E92582F84A
:041D83000222F8221E
:0C1D8700E6FC08E6FD08E6FE08E6FF2288
:0D1D9300E6FB08E6F908E6FA08E6CBF822C0
:101DA000BB010DE58229F582E5833AF5830222CF56
:101DB0005007E92582F8021D93BBFE07E92582F84A
:101DC0000222DBE58229F582E5833AF5830222E8E7
:0C1DD000ECF608EDF608EEF608EFF6223F
:0C1DDC00ECF0A3EDF0A3EEF0A3EFF0227A
:101DE800A8828583F0D083D082121DFF121DFF12B6
:101DF8001DFF121DFFE473E493A3C583C5F0C583DB
:101E0800C8C582C8F0A3C583C5F0C583C8C582C844
:011E180022A7
:101E1900BB010DE58229F582E5833AF58302231694
:101E29005007E92582F8022304BBFE07E92582F859
:101E3900022356E58229F582E5833AF58302236870
:101E4900BB0120E58229F582E5833AF583D0F0D0FC
:101E5900E0F8D0E0F9D0E0FAD0E0FBE8C0E0C0F06B
:101E690002234D5018E92582F8D083D082D0E0F9B9
:101E7900D0E0FAD0E0FBC082C08302230DBBFE187C
:101E8900E92582F8D083D082D0E0F9D0E0FAD0E019
:091E9900FBC082C08302235F221A
:101EA200D083D082F8E4937012740193700DA3A3CF
:101EB20093F8740193F5828883E4737402936860E3
:061EC200EFA3A3A380DFE3
:061EC8008A838982E473A5
:101ECE00E5132582F582E5123583F583B512048577
:101EDE0082132210AF06858213F51222858213F526
:041EEE0012D2AF223B
:0D1EF200E5132582F582E5123583F5832284
:10A3FE0090FDD21222A77810EC4D4E4F70047CA522
:10A40E007DA5C3EC13FCED13FDEE13FEEF13FF5011
:10A41E0010EC64CCFCED644CFDEE644EFEEF64CEAD
:10A42E00FFD8DF90FDD2121DDCEE547FFE2290FD90
:0DA43E00D2EEF0EFA3F0A374A5F0A3F0227E
:1064B000E508302C0104F823282467F582E434FB36
:1064C000F5832290FB64302C0390FB67E475F001A8
:1064D00012231F02193260EAC50C7002150B14C595
:1064E0000C202C04FF02B1A390FB6474FFF5F002B2
:1064F0002336FF02B033E5096006D509037F002289
:10650000202C0F12B01FEF6008050CE50C7002057F
:106510000B2290FB64122316121932FF60E890FBE5
:1065200064E475F00112231F80DC126500EFC0E007
:106530001264F2D0E040F3809DD22C8002C22C90F5
:10654000FB6412234DE4F50AF508F50BF50C75090B
:1065500000C22BC229C22AC22D1264C3FF7005AF2C
:106560000A7E0022B425301264C3FF24D0B40A008E
:10657000500C75F00AC509A42509F50980E924CF56
:10658000B41A00EF5002C2E502679ED22A80D8D228
:106590002980D4D22D80D0EF1264F2500812652ADF
:1065A000EF600E80A9EFC0E0126500D0E06F609E42
:1065B000EF60741264D680A7126500EF6069E50988
:1065C000700705098003126500EF6014202D0E127C
:1065D00064B0E475F00112231FEF12199AD509E691
:1065E000202D040508050A80BA1264F6EFC0E012F7
:1065F00064F2D0E050041264D6E4FF202D0E126441
:10660000B0E475F00112231FEF12199AEF70DA202F
:106610002D040508050A808BE5096002050912654D
:106620002A1264F6EF70C6302C04E41264D6E50A30
:10663000600302655F7EFF7FFF22202D1174FFFC47
:10664000FDFEFF1264B0122316121D4905080265F3
:106650004ED0E080D27900800A79108006790880D7
:1066600002790AD22EE50960020509E9C0E0126547
:106670002AEF60DD126500BF2D04D22B8003BF2BF3
:106680000912652AEF60CA1264F6D0E0B40A0280EB
:1066900033B40802802EBF302770027408C22EC0A7
:1066A000E01264F6D0E0BF78028003BF58160509F7
:1066B000D509028007D50904D22E800B74108019E9
:1066C0007002740ABF000AEFF8E4FCFDFEFF0267E7
:1066D00051C0E0EF1264D6D0E0F9E4FCFDFEFFE922
:1066E000C0E0ECC0E0EDC0E0EEC0E0EFC0E012645E
:1066F000F6EFF8D0E0FFD0E0FED0E0FDD0E0FCD037
:10670000F0E8604DB461004007B47B005002C2E580
:1067100024D0503DFA24F6500724F95034240AFAC4
:10672000EAB5F000502BCFA9F0A42FFF92D5E9C510
:10673000F0CEA4A2D53EFE92D5E9C5F0CDA4A2D557
:106740003DFD92D5E9C5F0CCA4A2D53CFCC22E807B
:066750008EE8C0E0202DE0
:106756002A202E08050A302B031222991264B01241
:106766002316050820290B202A0DEE8FF012227A17
:106776008009121D498004EF12199AD0E01264D6DE
:1067860002654E202D101264B01223160508E50B83
:10679600850CF012227A80E8121EA26618536659FA
:1067A60058658F4C658B42656748665D4F666144E8
:1067B60065B843665549666155663A46663A456622
:0C67C6003A4765932A67894E00006597EA
:101EFF00E3F5F009E208B5F06D606B80F3E3F5F000
:101F0F0009E608B5F060605E80F387F009E608B572
:101F1F00F054605280F487F009E208B5F04860464B
:101F2F0080F488828C8387F009E0A3B5F03860369F
:101F3F0080F488828C8387F009E493A3B5F027603F
:101F4F002580F388828C83E3F5F009E0A3B5F016C2
:101F5F00601480F388828C83E3F5F009E493A3B5D2
:101F6F00F004600280F202202A808580E7808E8054
:101F7F00D2803C8015806C807E809B80B5808B806A
:101F8F00A1804F8070803A02204089828A83ECFAC8
:101F9F00E493F5F0A3C8C582C8CCC583CCE493A362
:101FAF00C8C582C8CCC583CCB5F070606E80E1899E
:101FBF00828A83E493F5F0A3E208B5F05E605C805B
:101FCF00F289828A83E0F5F0A3E608B5F04D604B05
:101FDF0080F389828A83E0F5F0A3E208B5F03C60D4
:101FEF003A80F389828A83E493F5F0A3E608B5F08B
:101FFF002A602880F2805D89828A83ECFAE493F567
:10200F00F0A3C8C582C8CCC583CCE0A3C8C582C81D
:10201F00CCC583CCB5F004600280E27F00F845F0B8
:10202F00600EE863F0806480D395F01F40027F015B
:10203F002289828A83ECFAE0F5F0A3C8C582C8CC66
:10204F00C583CCE0A3C8C582C8CCC583CCB5F0CBC3
:10205F0060C980E389828A83ECFAE0F5F0A3C8C5F2
:10206F0082C8CCC583CCE493A3C8C582C8CCC58332
:10207F00CCB5F0A760A580E288F0ED2402B404008F
:10208F005099F582EB2402B40400508F232345822C
:05209F0023901F78737F
:10AFF600E4FFFE121932600C0FEF70010E09E970C2
:05B00600F20A80EF22B8
:1020A400E3F5F009E208B5F06BDFF58067E3F5F0DE
:1020B40009E608B5F05EDFF5805A87F009E608B551
:1020C400F052DFF6804E87F009E208B5F046DFF6FD
:1020D400804288828C8387F009E0A3B5F036DFF66E
:1020E400803288828C8387F009E493A3B5F025DFDE
:1020F400F5802188828C83E3F5F009E0A3B5F01420
:10210400DFF5801088828C83E3F5F009E493A3B5AE
:10211400F002DFF40221D3808780E9809080D480AC
:102124003E8015806E807E809D80B7808D80A380E8
:10213400518074803C0221DF89828A83ECFAE49323
:10214400F5F0A3C8C582C8CCC583CCE493A3C8C5A5
:1021540082C8CCC583CCB5F076DFE3DEE18070893C
:10216400828A83E493F5F0A3E208B5F062DFF48099
:102174005E89828A83E0F5F0A3E608B5F051DFF5C5
:10218400804D89828A83E0F5F0A3E208B5F040DF50
:10219400F5803C89828A83E493F5F0A3E608B5F0E0
:1021A4002EDFF4802A8002805789828A83ECFAE445
:1021B40093F5F0A3C8C582C8CCC583CCE0A3C8C539
:1021C40082C8CCC583CCB5F006DFE4DEE280007FB4
:1021D400FFB5F0020F2240027F012289828A83EC3C
:1021E400FAE0F5F0A3C8C582C8CCC583CCE0A3C887
:1021F400C582C8CCC583CCB5F0D5DFE5DEE380CF9E
:1022040089828A83ECFAE0F5F0A3C8C582C8CCC5FC
:1022140083CCE493A3C8C582C8CCC583CCB5F0AF46
:10222400DFE4DEE280A988F0EF60010E4E60ABEDE2
:102234002402B404005098F582EB2402B404005044
:0A2244008E232345822390211B7393
:10224E00EF4E6012EF60010EEDBB010B89828A83A7
:10225E00F0A3DFFCDEFA2289F05007F709DFFCA9B4
:0C226E00F022BBFEFCF309DFFCA9F0220B
:10A44B0090FD7FE0FFA3E0FEA3E0CF90FBC0F0A365
:10A45B00EEF0A3EFF090FD82E0CBF0A3E0CAF0A307
:10A46B00E0C9F07F2290FBC3AD82AC831219328D11
:10A47B00828C83F0A309E970010ADFEC90FD82E086
:0AA48B00FBA3E0FAA3E0F90261B0C0
:1096E9000251AAE493A3F8E493A34003F68001F29C
:1096F90008DFF48029E493A3F85407240CC8C33382
:10970900C4540F4420C8834004F456800146F6DF50
:10971900E4800B0102040810204080908C68E47EEC
:10972900019360BCA3FF543F30E509541FFEE49345
:10973900A360010ECF54C025E060A840B8E493A30C
:10974900FAE493A3F8E493A3C8C582C8CAC583CA37
:10975900F0A3C8C582C8CAC583CADFE9DEE780BEEF
:018D1B000057
:10227A00BB010A89828A83F0E5F0A3F0225006F7AF
:0F228A0009A7F01922BBFE06F3E5F009F31922AC
:0E229900C3E49FFFE49EFEE49DFDE49CFC2256
:0C22A700E0FCA3E0FDA3E0FEA3E0FF22AA
:0C22B300E2FC08E2FD08E2FE08E2FF2267
:1022BF00E493FC740193FD740293FE740393FF2265
:0C22CF00E0F8A3E0F9A3E0FAA3E0FB2292
:0D22DB00E2FB08E2F908E2FA08E2CBF82283
:1022E800E493F8740193F9740293FA740393FB224C
:0C22F800ECF208EDF208EEF208EFF22222
:09230400E6FB08E6FA08E6F922FE
:09230D00EBF608EAF608E9F622F5
:09231600E0FBA3E0FAA3E0F922C8
:10231F00F8E0FBA3A3E0F925F0F0E5821582700247
:07232F001583E0FA38F022EB
:10233600F8E0FBA3A3E025F0F9F0E5821582700230
:072346001583E038FAF022D4
:09234D00EBF0A3EAF0A3E9F02291
:09235600E2FB08E2FA08E2F922B8
:09235F00EBF208EAF208E9F222AF
:0C236800E493FB740193FA740293F922D1
:10614B00E50D24C0F582E434FBF583E0050D2290C8
:10615B00FBBD30270390FBC0E475F00112231F0237
:10616B0019322020E97F2ED2208018EF540F249073
:10617B00D43440D4FF30240BEF24BFB41A005003A7
:10618B002461FFE50E6002150E0511E51170020585
:10619B001030270E90FBBDE475F00112231FEF02A8
:1061AB00199A02ACAD7403D2278003E4C227F50D14
:1061BB0090FBBD12234DE4F50EF510F511E50E60C5
:1061CB00077F2012618E80F5750FFFC221C220C29E
:1061DB0022C223C225C226C22812615AFF700D307B
:1061EB0027057F0012619FAF11AE1022B4255FC24D
:1061FB00D5C22412615AFF24D0B40A00501A75F08C
:10620B000A780E30D50508B6FF0106C6A426F6207F
:10621B00D5047002D22380D924CFB41A00EF5004D6
:10622B00C2E5D2240263A0D22180C6D22080C0D284
:10623B002280BCD2D580BAD22580B47F2012618E49
:10624B002022077401B50E0040F112614BFF126161
:10625B008E0261C8D228D226809512614BFB126147
:10626B004BFA12614BF94A4B700679717A647BFFDA
:10627B0020222EE50E602A7E008E82758300121975
:10628B004B60060EEE650F70F0C2D5EBC0E0EAC0B6
:10629B00E0E9C0E0EE1263E7D0E0F9D0E0FAD0E03D
:1062AB00FB121932FF60AAEBC0E0EAC0E0E9C0E0E4
:1062BB0012618ED0E02401F9D0E03400FAD0E0FB7B
:1062CB00E50F0460DCD50FD980877BFF7A6379E318
:1062DB00D222809C791080027908C226C2288008BD
:1062EB00D2D5790A8004790AC2D5E50F047002F57C
:1062FB000FE4FAFDFEFF12614BFC7B082021131209
:10630B00614BFD7B1030200A12614BFE12614BFF7B
:10631B007B20EC3382D592D55013C3E43020069FFB
:10632B00FFE49EFEE42021039DFDE49CFCE4CBF8FE
:10633B00C221EC700CCFCECDCCE824F8F870F380F2
:10634B0017C3EF33FFEE33FEED33FDEC33FCEB33D2
:10635B00FB994002FB0FD8E9EB302105F8D0E0C4E4
:10636B0048B221C0E00AEC4D4E4F78207B0070C242
:10637B00EAB50F0040BCC0E01263E9D0F0D0E020DA
:10638B002104C4C0E0C4B221C0F0126177D0F0D5B3
:10639B00F0EB0261C8121EA262655362DF586236CF
:1063AB004C62324262E34F62EB4462EB49624B4315
:0863BB0062F15562D54662D57E
:1063C3004562D547649150623A2D623E2E62612B3D
:1063D300624223625F20647A2A61FA4800006259AC
:1063E3003F3F3F00790AA2D5202314302509B91075
:1063F300020404B9080104A2D52026025001042096
:1064030022689222B50E005034C0E07F2030231959
:106413007F30A22272267225500F126440C222C21C
:1064230026C225C2287F30800F302503E9C0E01241
:10643300618E302503D0E0F9D0E0B50ECC302517BE
:106443007F30B9100C12618E7F583024077F78801B
:1064530003B9080312618E3022057F2D02618E7FFE
:10646300202028F87F2B2026F322922280CF286E2B
:10647300756C6C2900D22112614B3021F8C221784E
:106483000E30D50108F60261FA2D504349581261C6
:106493004B2403B405004001E490648C9312617FA4
:0D64A300743A12617FD223750E040262DF8D
:10B01F0010330B12B180BF0D027F0A02ACAD90FE50
:04B02F0065E0FF22B7
:08B1A30090FE65EFF0D23322AB
:10B03300EFC394094005EF940E4004EFB42003D30B
:04B043008001C322A3
:10ACAD00EFB40A07740D12ACB8740A309811A89954
:10ACBD00B8130CC2983098FDA899C298B811F63007
:07ACCD0099FDC299F59922DF
:0AB180003098FDAF99C2987E0022BE
:00000001FF
